:1090E200414952434F54454300405621332E3130BB
:1090F20020454E4700424154540042414400403210
:1091020044400040334440004F4646214E455740BC
:109112004D454E55000A16000180000300007E00F6
:1091220000FE00001E0000360003E60001C400003D
:1091320000000FFFE053454152434840534154530E
:109142000043414C40414C544920202300504943A4
:10915200545552450052414E4B494E47004D4150E5
:109162002020200043454E54455200564152494F5B
:1091720020004241524F475200524F55544553002E
:109182004E454152535400574159505453004D419A
:10919200524B53200044454641554C540020202058
:1091A2002141564721202020204453540021455874
:1091B20049540153454C40524F555445015345546F
:1091C2002048454947485401464C49474854532092
:1091D2006869015741595054532020686901524F20
:1091E2005554455320206869014149525350414327
:1091F2004568690153455454494E475368690053C1
:10920200455420484549474854004241524F40483E
:109212004549474854004750532048454947485418
:1092220000514E4820202020402148504100464C09
:10923200004C4F47424F4F4B20454D505459003E32
:109242002145584954002145584954015245504C32
:1092520041590153454E440144454C455445002172
:109262004558495401544E432031232035374B0190
:10927200544E4320312320392E36010150574340AA
:109282003130234035374B01505743403130234072
:1092920031394B01014D5850403130234035374B65
:1092A200014D58502034232035374B014D58502062
:1092B20031232035374B014D585040313023403156
:1092C200394B014D58502034232031394B014D5830
:1092D200502031232031394B002145584954014E49
:1092E200455720205741595054014544495420576D
:1092F200415950540144454C202057415950540182
:1093020001434F4D3A015245434549564520575076
:109312000153454E442057415950540153454E4440
:1093220040414C4C4057500101444953542057503E
:109332002D57500144454C40414C4C40575054002D
:109342004252472021444953540053544F5245003E
:1093520050524553454E5440504F532E00555044A1
:109362004154494E472E2E004044454C45544544F5
:1093720000534552200049524441005553422000B7
:1093820020425420004C4953540053454E4400207F
:109392005452414E534D4954204552524F5220008F
:1093A20021455849540153454C40524F55544501AB
:1093B2004E455720205254455054014544495420AB
:1093C200524F555445015245564552534520525429
:1093D2000144454C202052544550540144454C20F0
:1093E20020524F5554450101434F4D3A01524543D6
:1093F200454956452052540153454E4420524F553B
:1094020054450053454C21524F555445004E40455A
:10941200405700204E455740504F534021002140B5
:10942200524556455253454000524556525300212B
:109432004044454C405750545300214044454C2031
:10944200525445004E4F5420454D5054592000214E
:0D9452004053454E444052544500214558BA
:10945F004954014C4F41444043545221504301560B
:10946F00494557404354520144454C40414C4C21CF
:10947F004354520101434F4D3A0152454356202068
:10948F004354520153454E442020435452005649F1
:10949F004557204354520020204D4F564500202061
:1094AF004D4F564520544F005343414C45202058B3
:1094BF002F5920204558495400434C5220444953BA
:1094CF0054004155544F43454E54004155544F207D
:1094DF004F4646002020205343414C4500444953FA
:1094EF0054204B4D0044495354204E4D00214558B4
:1094FF00495401564152494F202020686901584371
:10950F002D53455420206869015254452D5345541D
:10951F002068690147454E4552414C20686901500A
:10952F004943545552455368690101014541535907
:10953F002D53455401464143544F525953455401FD
:10954F0044454D4F464C494748540144454C2141F1
:10955F004C4C21464C490021455849540153494E22
:10956F004B544F4E450153494E4B212D0153494EFC
:10957F004B404D4F440153494E4B40494E560156B7
:10958F004152205443402020402301564F4C554D0B
:10959F004501564152494F204E554C4C01534F55A2
:1095AF004E44014652455155454E5A01564152209F
:1095BF004156402030402301544543202020403065
:1095CF0030402501534F554E44434845434B0053BC
:1095DF00494E4B21544F4E450053494E4B54214F4A
:1095EF004646004E4F542150524553454E54005657
:1095FF004152494F204E554C4C004B454550405120
:10960F0055494554403130404D494E004245464F33
:10961F005245204E554C4C494E4700214558495410
:10962F00014D415021545241434B014155544F4339
:10963F00454E5401014156472F4449535401474C5D
:10964F00444550415448014C2F44010157494E4461
:10965F0021542D55500143454E5421542D55500042
:10966F0021455849540153544152544054494D4592
:10967F000146495253540144454C544120203A016C
:10968F004D554C5449504C45014C415354010153D5
:10969F00454C40524F5554450101010143594C521D
:1096AF000143594C20542D55500021455849540120
:1096BF0001554E495401434C49434B40302C4020F7
:1096CF002301434F4E5452415354014E4D454121B6
:1096DF0031383301494D50454C4C455200405741AC
:1096EF0059504F494E5420455849535453400057F1
:1096FF004159504F494E540020204558495420207D
:10970F0021005245434549564500465245454000C4
:10971F004E455854205450540050524556205450E2
:10972F005400434C5220404C454700434C5220407C
:10973F0053554D004F46462020202020202020004A
:10974F00204F464600475053204552524F52005328
:10975F00544F52494E4700524F555445004E4541C4
:10976F0052455354004C4953542000455445004131
:10977F004C54403000454D50545920525445200010
:10978F0020544F4F404D5543482000214053454CE6
:10979F00404C495354002053454C4057505440219E
:1097AF000021405245434549564540002020404F37
:1097BF00204B40202021004F4B0020204641494C98
:0D97CF002020210020455849540045444900
:1097DC0054005940454053004544495420204E45BF
:1097EC0057202053544F5245004E45585420534552
:1097FC004C4543542045584954005843542D464C2D
:10980C004947485420005553454400454E54455251
:10981C0020004D4D2E4D4D4D20004D4D2753532EB8
:10982C005300574753213834002040554054404D85
:10983C00402000554054404D002055544320004CCE
:10984C004F43414C005357495353474400414C54E8
:10985C0000535549405800415647402030402300A2
:10986C00353030003136343000205D203130404B03
:10987C00632F70005D2020203140632F2300205D7A
:10988C00202035404B5453005D2032303040465040
:10989C004D00406340204B63004654204B63004016
:1098AC006340204E4D004654204E4D004D2F53002A
:1098BC003230305E003530305E0031220032220012
:1098CC00332200352200382200464C3700464C31FA
:1098DC003600464C333300464C363500463130307A
:1098EC0000463136300046323630005E2526405375
:1098FC004F47005E25264054415300414C540056BE
:10990C00415200225E2F24004B545300532F4E0023
:10991C002224004B5400225E004E4D00302C3500AA
:10992C00312C3000322C3000302C3600312C3200EF
:10993C00322C3500332C3800372C350040313500B3
:10994C00403330004036300020545241434B214FBD
:10995C004E20200020545241434B214F46462000BC
:10996C003C2D204C495354202D3E20204558495421
:10997C000053454C004E455854005441534B00463F
:10998C004C2D4441544500545000544F4600535400
:10999C00410046494E004C414E00534554204F4621
:1099AC0046534554004953412048454947485400C3
:1099BC004D41524B0020545241434B2D55502120C8
:1099CC0000204E4F5254482D5550212000564152E4
:1099DC0000464958004741544521580053544152C0
:1099EC00544C494E452000535443594C2000404F91
:1099FC0046460054502000406A40494E20004067C3
:059A0C00404F5554001D
:10497600304D2475A7049005C2E0F51CE0F51DE056
:10498600F51EE0F51FE0F56DE0F56EE0F56FE0F57C
:1049960054125538124F762275C70375C6E475B999
:1049A60001E5BCB48143125538125F428E628F63B3
:1049B6007568F9756900124A4C203C2D203B2B1274
:1049C6004B81124B55856D1C856E1D856F1E85545A
:1049D6001F124AB8203C12203243201D23124B815D
:1049E600124F76E532242850DC22124AB8203CF9D0
:1049F600203DF6203205201DBD80EF301DB880EA2F
:104A0600124B81124F76856D1C856E1D856F1E8536
:104A1600541F124B6B124F76203DCE8099124DA437
:104A2600201D0D7553107400124D07203DBB808666
:104A3600E553540FC553C4540F203505124C1C8042
:104A460003124D07808BC23CD23B124B08FD124B22
:104A560008FC124B08C39573F565EC9574F564ED87
:104A66009575600504600A800EE56424E0501180A7
:104A760006E56424204009124B08124B08024B0835
:104A8600124B08FD124B08FC124B08C39576F567CE
:104A9600EC9577F566ED9578600904600122E56688
:104AA600F48002E5668562F0A474E025F04002C257
:0D4AB6003B22C23C124B08A2E7923DA2E653
:104AC300921DA2E592324026A2E492E592E692E795
:104AD300FC124B082565F565EC3564F564124B084B
:104AE300FC124B082567F567EC3566F56622A2E4F0
:104AF3009235540F79C6F7124B0809F7301D05128A
:104B03004B08F55322E5697023E5686030240340C0
:104B13002CE56875F004A485F0C7F5C675B901E501
:104B2300BCB4811985BD68756902801E5403701079
:104B330005C675B901E5BC056953690F22D23C224C
:104B4300147004E5BD80F0147004E5BE80E9E5BF90
:104B530080E575A7009006F6E56DF0A3E56EF0A37A
:104B6300E56FF0A3E554F02275A7009006F6E0F593
:104B73006DA3E0F56EA3E0F56FA3E0F55422E564C1
:104B8300B2E7F56D85656EAB67E566FC30E707C395
:104B9300E49BFBE49CFCAA62A963125C5CE56630BF
:104BA300E707C3E49DFDE49EFEEEB2E7F56F8D5487
:104BB3002275380C124E0D124E58D55301227538FA
:104BC3000C124DDE124E4ED5530122753800124D94
:0E4BD300F6124E1DD5530122753800124DDE2C
:104BE100124E1DD5530122753803124E0D124E89F6
:104BF100D5530122753803124DDE124E7FD5530174
:104C01002275380F124DF6124EAED553012275386A
:104C11000F124DDE124EAED5532622904C21237336
:104C21008091807780688059804A803B802C801DEC
:104C3100800E80DA80CB80BC80AD809E808F8080AA
:104C4100753815124E0D124ED0D5530122753815F7
:104C5100124DDE124EC5D5530122753809124DF69B
:104C6100124E96D5530122753809124DDE124E9619
:104C7100D5530122753806124E0D124E40D55301FF
:104C810022753806124DDE124E35D5530122753884
:104C910012124DF6124E66D5530122753812124D7D
:104CA100DE124E66D5530122024BB4753815124EF1
:104CB1000D124ED0D553012275380F124DDE124E12
:104CC100AED553012275380F124DF6124EAED553A3
:104CD1000122753803124DDE124E7FD55301227524
:104CE1003803124E0D124E89D55301227538001228
:104CF1004DDE124E1DD5530122753800124DF612AC
:104D01004E1DD5532622904D0C2373809E80A98081
:104D1100B480BF80CA80D580E08010801B8026804F
:104D210031803C80478052805D806875380C124D1F
:104D3100DE124E4ED553012275380C124E0D124E15
:0E4D410058D5530122753812124DDE124E66FF
:104D4F00D5530122753812124DF6124E66D5530106
:104D5F0022753806124DDE124E35D55301227538A5
:104D6F0006124E0D124E40D5530122753809124DC1
:104D7F00DE124E96D5530122753809124DF6124E9A
:104D8F0096D5530122753815124DDE124EC5D553E7
:104D9F000122024CAC78C686040886037AED125CB9
:104DAF001A78CAA60408A60378C686040886037A6A
:104DBF0062125C1A78CCA60408A60378C68604088B
:104DCF0086037AB5125C1A78C8A60408A603227562
:104DDF001A6A751B0A78CA86180886191250217824
:104DEF00CC86060886072278C88618088619E4F547
:104DFF001AF51B12502178C886060886072278C636
:104E0F008618088619751A00751B01025021E51DB9
:104E1F002519F51DE51C3518F51CC3E51F9FF51F5A
:104E2F00E51E9EF51E22C3E51F9FF51FE51E9EF58D
:104E3F001EC3E51D9519F51DE51C9518F51C22E5FA
:104E4F001D2FF51DE51C3EF51CC3E51F9519F51F1C
:104E5F00E51E9518F51E22C3E51D9FF51DE51C9E49
:094E6F00F51CC3E51F9519F51FA0
:104E7800E51E9518F51E22E51F2FF51FE51E3EF5C8
:104E88001EE51D2519F51DE51C3518F51C22C3E581
:104E98001D9519F51DE51C9518F51CE51F2FF51F27
:104EA800E51E3EF51E22E51D2FF51DE51C3EF51CF1
:104EB800E51F2519F51FE51E3518F51E22C3E51D4A
:104EC8009FF51DE51C9EF51CE51F2519F51FE51E20
:104ED8003518F51E22E51A7009E51B70058C068D3C
:104EE8000722ED851BF0A4A2F792D5ED851AF0A450
:104EF800AEF0FFEC851BF0A4A2D53FEE35F0FF9293
:104F0800D5EC851AF0A42FFFE435F030D50104FE66
:104F180022E4F51AF51BEF4E7003051B22EF651905
:104F28007006EE65187001227808C3EF33FFEE3380
:104F3800FEEF9519F5F0EE95184003FEAFF0E51A6F
:104F480033F51AD8E5F4F51A751BFF7805C3EF3366
:104F5800FFEE33FEEF9519F5F0EE95184003FEAF1E
:034F6800F0E51B56
:104F6B0033F51BD8E5F4C403F51B22E51D9511E5BC
:104F7B001C9510500BE56E9511E56D9510500122A7
:104F8B00E51F9511E51E9510500BE5549511E56F36
:104F9B009510500122E51D9513E51C9512400BE56C
:104FAB006E9513E56D9512400122E51F9513E51ED5
:104FBB009512400BE5549513E56F95124001225362
:104FCB002CF8C3E51F9554FFE51E956FFE926050BC
:104FDB0007C3E49FFFE49EFEC3E56E951DF519E53F
:104FEB006D951CF5189261500BC3E49519F519E4F6
:104FFB009518F518C3E5199FE5189E9262500AE5BE
:10500B0018CEF518E519CFF519124F19E52C5407E1
:10501B0075F003A4F538E5389050277302503F0222
:10502B00505302506102507902508C02509F025033
:10503B00AD0250C5851C16851D17C3E4951FF515CC
:10504B00E4951EF5140250D8851C16851D17851E78
:10505B0014851F158077C3E4951DF517E4951CF592
:10506B0016C3E4951FF515E4951EF514805FC3E494
:05507B00951DF517E48E
:10508000951CF516851E14851F15804CC3E4951FCD
:10509000F517E4951EF516851C14851D15803985B8
:1050A0001E16851F17851C14851D15802BC3E495BE
:1050B0001FF517E4951EF516C3E4951DF515E49547
:1050C0001CF5148013851E16851F17C3E4951DF566
:1050D00015E4951CF5148000C3E5179513E51695A6
:1050E0001210D70122E5159513E514951210D7017A
:1050F00022E519F92517FFE518F83516FED3EF95C7
:1051000011EE9510500122E5119517FDE510951649
:10511000FC402A4D6027124EDDE5152FF515E514EC
:105120003EF514E5159513E514951210D70122E507
:10513000199DF9E5189CF8851016851117E51729B2
:10514000FFE51638FEE5139FE5129E500BC3E513ED
:105150009517F9E5129516F8E51A700AE51B700621
:10516000AA00AB018013E9851AF0A4E5F0FBE885FD
:105170001AF0A42BFBE435F0FAE5152BFBE5143A05
:06518000FAE5119BE510A9
:105186009A10D70122EB9515FDEA9514FCC3E51597
:105196009511E514951010D717E5139BE5129A5053
:1051A60036E5139515FFE5129514FE125455802722
:1051B600EB9511FFEA9510FEAA00C001125455D0D6
:1051C60003E5172BFBE5163AFAEB99F517EA98F57E
:1051D60016851115851014C2D5E5466002D2D5AAEA
:1051E60056E98AF0A4ABF0E88AF0A42B30D5047512
:1051F600F00384F8700122E5172513FDE516351234
:10520600FCED8AF0A4ABF0EC8AF0A42B30D5047543
:10521600F00384FEE5152513FDE5143512FCED8A31
:10522600F0A4ABF0EC8AF0A42B30D50475F003841F
:10523600F9E53890523D7302525502526102526AA4
:1052460002527302527902528502528C025291C363
:10525600743E9EFFC3743E99FE8032C3743E9EFF29
:10526600AE018029AF06C3743E99FE8020AF06AE1C
:0D52760001801AC3743E9EFEC3743E99FF72
:10528300800EC3743E99FF8007C3743E9EFEAF0138
:1052930008EF2437FFE51B7007E51A700CE8800E52
:1052A300A2E7E51A50030460F488F0A4E5F0600176
:1052B30004F923FA98FBC3E998C333F99052C5E57F
:1052C30038730252DD02530A02533F02536C0253F6
:1052D300990253C60253F302542005A7800BEB3007
:1052E300E7032A8002291E1FFBEEC45403F583EE55
:1052F3005408C42FF582EE5407243883F5F0E045B3
:10530300F0F0D8DA05A72205A7800BEB30E7032AD4
:105313008002290E1FFBEEC45403F583EE5408C428
:105323002FF582EE5407240B83F5F0E045F0F0D817
:10533300DA05A722804020100804020105A7800B8C
:10534300EB30E7032A8002291E0FFBEEC45403F55A
:1053530083EE5408C42FF582EE540724EC83F5F052
:10536300E045F0F0D8DA05A72205A7800BEB30E77C
:05537300032A8002295D
:105378000E0FFBEEC45403F583EE5408C42FF582D8
:10538800EE540724BF83F5F0E045F0F0D8DA05A71E
:105398002205A7800BEB30E7032A8002291F1EFB9A
:1053A800EEC45403F583EE5408C42FF582EE540777
:1053B800249283F5F0E045F0F0D8DA05A72205A796
:1053C800800BEB30E7032A8002291F0EFBEEC45442
:1053D80003F583EE5408C42FF582EE540724658341
:1053E800F5F0E045F0F0D8DA05A72205A7800BEB29
:1053F80030E7032A8002290F1EFBEEC45403F5830D
:10540800EE5408C42FF582EE5407243883F5F0E0F3
:1054180045F0F0D8DA05A72205A7800BEB30E703A3
:105428002A8002290F0EFBEEC45403F583EE5408BC
:10543800C42FF582EE5407240B83F5F0E045F0F015
:10544800D8DA05A7228040201008040201EC701F5A
:08545800ED20E740D2E023CF74
:1054600023CF30E7F980357B08801A7B1080167BCC
:105470002080127B40800E20E4ED20E3EE20E2EF5E
:1054800020E1F07B80EE8BF0A4CF8BF0A4E5F02F31
:10549000FFEC8BF0A4CD8BF0A4E5F02D2499838F45
:1054A000F0A433E5F033FBE98BF0A4E5F0C88BF012
:1054B000A428F9E435F0F822FFFEFCFAF8F6F4F23D
:1054C000F0EFEDEBEAE8E6E5E3E1E0DEDDDBDAD99B
:1054D000D7D6D4D3D2D0CFCECCCBCAC9C7C6C5C4F9
:1054E000C3C1C0BFBEBDBCBBBAB9B8B7B6B5B4B313
:1054F000B2B1B0AFAEADACABAAA9A8A8A7A6A5A4FF
:10550000A3A3A2A1A09F9F9E9D9C9C9B9A999998C2
:105510009797969594949392929190908F8F8E8D69
:105520008D8C8C8B8A8A89898887878686858584F5
:10553000848383828281818075A70090555EE546D1
:10554000FA24FA50027A05EA2323F978107F0493AB
:10555000F60809E9DFF9905576EA93F556227FC2FD
:10556000803E7F4680BA7E8C81747D1882E87A30D6
:1055700085D074608BA08080402010081255820274
:1055800057D8D215D274D273C219C23A125F428E62
:1055900047757D007546057552021285BE12021FC1
:1055A000E53524EB500E1285BE7F199094C8126B1E
:1055B000F712CFDCE55275F016A4F57012578E7510
:1055C00051151256597F237E099094A6126C091228
:1055D000CFDC10000810010D10021280E2125701FA
:1055E00075330180DA12574675330180D275510048
:1055F0001256597E009094B7126C3C7F237E059022
:1056000094AD126C091256AA12CFDCE55210000FAD
:1056100010010510028780D5045403F55280CE1284
:1056200056597F237E0B9094E5126C09E54660077E
:1056300014600414123C3A12CFDCE5461000081046
:10564000010B10021180D860D6154680D2B4050235
:1056500080CD054680C902559D75320012D19C7FD0
:10566000017E1190949D126C3C7E0012C7F6E551AC
:10567000D26612C84D75170812CC84123C7275712F
:1056800000C20612C99D741BFFF5177E0F9094ECA3
:10569000305D039094F4126C3C1286011264FE1289
:1056A000419BC20612499E02189CE5526014146088
:1056B0001E1460297F647E2D791C1256F41E1FD99A
:1056C000F9227F6A7E1F79281256F41FD9FA227FA9
:1056D000487E2D791C1256F40F1ED9F9227F567E72
:1056E0003379281F12D0E10F0F12D0E11F12D0E141
:1056F0001ED9F0221E12D0E10E0E12D0E11E02D0F1
:10570000E1E552605514606814606D800075709E0C
:1057100012577B8003757000E5732540F573E435FF
:1057200074F574E43575F575227570161257188086
:105730000375702DE5762542F576E5773541F577E9
:10574000E43578F57822E55260CB1460DC1460E132
:105750008000757044125734800375705AE5739554
:0957600040F573E5749400F57442
:10576900E5759400F5752275707112575D800375A2
:105779007088E5769542F576E5779541F577E57890
:105789009400F57822E5469057A493F540FEAD477D
:10579900E4FFFC125CEF8E418F4222020C1830604C
:1057A900C07F401209A51218B212CFDC125A4EEB73
:1057B900700590923A800B1258619097BB500390F4
:1057C90097C97F3F7E04126C0912CFDC12D0681290
:1057D900D09875370990945C12179D9057E8730219
:1057E90002970259A802557C025A7F0257D80258DB
:1057F900000258190257AA7F2E12113280D17F3622
:105809007E0490978F126C0912CFDC12D06880BF8A
:105819007F371209A51218B212CFDC125A3212437D
:105829001BD2AC1000A9306DFA125911203BCF40A0
:10583900ED7568F975160012595E40FB125AFA7F28
:10584900367E29E51612C5D412CFDC0516126CAFC7
:1058590078C6B6F7E2025A2C7C0512431B12CD8694
:10586900744112CDB9745312CD54EB12CD75126C2B
:10587900C15003DCE5227515F975160010000EE517
:105889001560251258B340051258DA5002D3227F09
:105899003F7E29E51612C5D412CFDC7F1412D07FC2
:1058A9000516E51664F870D4C32212723275B9016F
:1058B900E5BCB4811AE5BDF51570037516F778C610
:0B58C900A61612737B12737312737328
:1058D400C3027373D3227F0575F019D5E0FDD5F0AB
:1058E400FA12431B12CD86744112CDB9744212CD03
:1058F400547E0F78C6E60812CD54DEF912CD781224
:105904006CC1400122DF012275F00080CEC23B123F
:10591400431BD2AC12CEE6204C3CB440F712CEEB83
:10592400B4400312CEEBB4412DF53812CEEBB45390
:105934002512CEEBFA12CEEBE538701A12CEEBB488
:105944000D1412CEEBB40A0EC3E5169A4003026C92
:10595400A6C2ACD23B22C2ACD322126D0512431BA9
:10596400D2AC1000F112CEE6204CEBB440F412CECF
:10597400EBB4400312CEEBB441DCF53812CEEBB4F9
:1059840042D47E1078C612CEEBF608DEF9E5387004
:10599400C512CEEBB40DBF12CEEBB40AB9C2ACC380
:1059A400220257D87F0A1209A51218B212CFDC12AC
:1059B4005A3212436DD2AC1000E712CEEBB440F56C
:1059C400F53812CEEBB46EED12CEEBE538600A1268
:1059D400436D744F12CD6080DC12CDB4E51612CD48
:1059E4006012CD6A7568F975160012436DD2AC1059
:1059F400003912CEEBB440F7F53812CEEBB44EC5F5
:105A04007E1078C612CEEBF608DEF912436DE53847
:105A14006007744F12CD6080D1125AFA0516745182
:105A240012CD6078C6B6F7C2125A9B0257D87515C4
:0C5A34000075160412722975B901E5BC5A
:105A400030E70205160515E515242050EB227B00F2
:105A50007515F912723275B901E5BCB481010B05F7
:105A600015E515240350EC75150112722975B9015D
:105A7000E5BCB481010B0515E515242050EC227F0F
:105A80001C1209A51218F512CFDC10000B10010230
:105A900080F87515F9125A9B0257D8E5156037241E
:105AA00003401A241E5019E51524074002802712CE
:105AB0007232125AD70515E515240350F2751501F7
:105AC00012722975B901E5BC30E703125AD70515E2
:105AD000E515242050EA22125AEC1248EB05C612B2
:105AE00048EB05C61248EB05C60248EB74FF80017F
:105AF000E4F5BCF5BDF5BEF5BF22E568606AF515B5
:105B00000515E5152403501D75150112722975B987
:105B100001E5BC30E70280190515E515242050EB9E
:105B2000751500800C241D60F750E0E51524065023
:105B300037E56875F004A485F0C7F5C675BC81E546
:105B400015F5BDF56878C6B6F70375BD0008125B9C
:105B50005D125B57125B5786BC0886BD0886BE087F
:095B600086BF081248EB05C622BD
:10B3FF0012A22E12B4FE12774512B48312774D1299
:10B40F00B49002A23212A22E12B4FE1277457F5AC6
:10B41F00C23C127627127823783F79437F607EEA09
:10B42F0012B4F212774D7F65127627127823783D8A
:10B43F0079417F207E4E12B4F2303C2012B6B41206
:10B44F00B50F783F794312B46E783D794112B46EDF
:10B45F0012B6B478D7E65480F67537000287D3C397
:10B46F00E796FF1819E796FE0809C3E69FF7181924
:10B47F00E69EF7227F5B7E0690985D126C3C1F80E4
:10B48F000A7F667E14745912C6ED1F1274B07E398E
:10B49F00E402C70C7866E620E73418C3E694720816
:10B4AF00E694045029C318E6941F08E69404401E3E
:10B4BF007869E620E71818C3E6940E08E694015061
:10B4CF000DC318E6947508E694004002D322C322F8
:10B4DF00E67D0030E7011D08E62BFB18E63CFCE497
:0EB4EF003DFD22C3EB9FF6F71819EC9EF6F711
:10B4FD002212B4A3400CE47842F608F67840F60820
:10B50D00F6227864C3E6946AF55708E6944CF5562E
:10B51D000808C3E69458F55B08E694AEF55A7539FC
:10B52D0000AC56AD57EC12A5DB784C12A669AC5A9F
:10B53D00AD5BEC12A5DB785012A6697F2B7E867D64
:10B54D00777C1812A5A0785012A65D12A4AC12A596
:10B55D00A0785012A65D12A4AC12A5A0785012A628
:10B56D005D12A4AC12A5A07F367E847D257C64126D
:10B57D00A5A0785012A65D12A4AC12A5A0784C120D
:10B58D00A65D12A4AC12A5A07F3F7EA27D607C8B30
:10B59D0012A5A0785012A65D12A4AC12A29A12A206
:10B5AD009A12A6757F3F7E807D057CE6053912A433
:10B5BD00AC784812A6697F2C7E937D477C7F12A5BF
:10B5CD00A0785012A65D12A4AC12A5A0785012A6B8
:10B5DD005D12A4AC12A5A0784C12A65D12A4AC12FB
:10B5ED00A5A07F357EB47DF87CDF12A5A078501222
:10B5FD00A65D12A4AC12A5A0785012A65D12A4AC43
:10B60D0012A5A07F3F7EED7D227CCD12A5A0784CAA
:10B61D0012A65D12A4AC12A29E12A29A784412A692
:10B62D00697F317E397D9D7CE712A5A0784C12A6ED
:10B63D005D12A4AC12A5A0784C12A65D12A4AC129A
:04B64D00A5A07844F8
:10B6510012A65D12A29E12A5A07F2C7E377D0C7CC6
:10B66100A312A5A0784C12A65D12A4AC12A5A078D5
:10B671004C12A65D12A4AC12A5A0784C12A65D12C4
:10B68100A4AC12A29E12A6757F3F7E807D027C9F94
:10B69100053912A4AC784412A669784812A65D1245
:10B6A100A6128E428F43784412A65D12A6128E40D6
:10B6B1008F4122753900AC42AD43EC12A5DB7848CD
:10B6C10012A669AC40AD41EC12A5DB784412A66923
:10B6D1007F2B7E537D507C0912A5A0784812A65D70
:10B6E10012A4AC12A5A0784812A65D12A4AC12A5B2
:10B6F100A0784412A65D12A4AC12A5A07F347EF2FC
:10B701007DCD7CA312A5A0784812A65D12A4AC122F
:10B71100A5A0784812A65D12A4AC12A5A07F3F7E19
:10B721000A7D2E7CAE12A5A0784412A65D12A4ACAF
:10B7310012A29A12A29A784C12A6697F2B7E4F7D93
:10B74100AF7CB212A5A0784812A65D12A4AC12A5D6
:10B75100A0784812A65D12A4AC12A5A0784812A642
:10B761005D12A4AC12A5A07F357EB17D4B7C9512F4
:10B77100A5A0784812A65D12A4AC12A5A078441227
:10B78100A65D12A4AC12A5A07F3F7E497DCD7C456C
:10B7910012A5A0784812A65D12A4AC12A29E12A214
:10B7A1009A785012A669784C12A65D12A6128D5590
:10B7B1008E568F57785012A65D12A6128D598E5A49
:04B7C1008F5B7864BE
:10B7C500E557246AF608E556344CF608E555340481
:10B7D500F608E55B2458F608E55A34AEF608E43574
:03B7E50059F622F0
:1086210012A22E128CB212A2327F6690983F126C67
:108631003A12868F7F5A78C412866B12867378C677
:1086410012866B1286567F6578C812866B12867306
:1086510078CA12866B7E2DE51B12C70C7E33E51A94
:1086610012C70C7E39E51902C70C8604088603027D
:108671005BB97E15E51C12C70C7E1BE51B12C70CEE
:108681007E21E51A12C70C7E27E51902C70C7F5A15
:108691007E01E53A12C6227E0B9090A6E53B93023D
:1086A100C71FE6FF08E6FE08E6FD339217E4500116
:1086B100F4FC12A68675130A75390112A88478D7BD
:1086C100E6C2E775F00A84F9303D02A9F012A686E8
:1086D1008913053912A85D30170A053912A87005EA
:1086E1003912A870A80302A66912A22E128CB2C276
:1086F1003C7F5A7E031279D412868F12CFDC100090
:108701000810011510022080EFE53A146004153AB3
:108711008003753A3CD23C80DFE53AB43C05753ABA
:108721000180F2053A80EE7E031279CF7E0B127939
:10873100D412868F12CFDC10000810011510022010
:1087410080EFE53BB40205753B158002153BD23C39
:1087510080DFE53BB41505753B0280F2053B80EEF9
:108761007E0B1279CF7F5A78C412866B12867312F0
:0787710087DC12783378C4A5
:1087780012883478C612866B12865612880E751CBB
:108788000012783378C61288347F6578C812866BF1
:108798001286731287DC12783378C812883478CA44
:1087A80012866B12865612880E751C001278337862
:1087B800CA128834303C14E53B24F4500B78C9E6DF
:1087C8002410F618E63427F612883A12A2321273E9
:1087D800B502CFDCC2247E15E51C127924F51CD223
:1087E800247E1BE51B127924F51B1023E77E21E567
:1087F8001A127924F51A1023E67E27E5191279242E
:10880800F5191023E822C2247E2DE51B127924F5E0
:108818001BD2247E33E51A127924F51A1023E77E39
:1088280039E519127924F5191023E622ECF608EB3C
:10883800F6221290BE78C8E6FE0886073395E0FD5A
:10884800FC12A5A07FE87E037D007C0012A884129C
:10885800A5A078CAE6FE0886073395E0FDFC12A8B5
:108868005D12A5A07F807E697D677CFF12A85DEC04
:1088780012A5D712A5A07F3F7E807D0D7C1D12A476
:10888800AC12A5A07F3D7E407D007C0012A5A0789B
:10889800BC12A65D12A4AC12A5A07F3E7E807D000E
:1088A8007C0012A29E12A5A078BC12A65D12A4ACF0
:0988B80012A5A07F3F7E807D0027
:1088C1007C0012A29A12A5A078B412A65D12A4ACE3
:1088D10012A524783C12A6697F407E807D007C0031
:1088E10012A5A0783C12A65D12A4AC12A70312A592
:1088F100A07F3F7EA87D007C0012A5A078B812A6BB
:108901005D12A4AC12A4AC12A5A07F407E007D0034
:108911007C0012A5A0783C12A65D12A4AC12A7039C
:1089210012A5A07F3F7EC07D007C0012A4AC12A2E4
:108931009E12A5A078B812A65D12A4AC12A5A078CB
:108941003C12A65D12A29E785412A66912A6ED7879
:108951005812A66912A5A012A4AC12A5A078C01243
:10896100A65D12A4AC784412A669785412A65D12D1
:10897100A703783C12A66912A5A012A4AC12A5A067
:1089810078BC12A65D12A4AC783C12A6697F3E7E2B
:10899100C07D007C0012A5A0783C12A65D12A4AC9B
:1089A10012A5A07F3F7E007D007C0012A29E12A531
:1089B100A0783C12A65D12A4AC12A5A07F3F7E80D8
:1089C1007D007C0012A29E12A5A078B412A65D12B1
:1089D100A4AC787012A66978C4E6FE0886073395C0
:1089E100E0FDFC12A5A07FE87E037D007C0012A8BB
:1089F1008412A5A078C6E6FE0886073395E0FDFC43
:108A010012A85D12A5A07FE07E5E7DF87CFF12A812
:108A11005DEC12A5D712A5A07F3F7E7F7DE57CC9C5
:058A210012A5A0787011
:108A260012A65D12A4AC12A524785012A6697F3F47
:108A36007EF07D007C0012A5A0783C12A65D12A4F3
:108A4600AC12A5A07F3F7EC07D007C0012A29E12C4
:108A5600A5A0783C12A65D12A4AC12A5A07F3F7E0D
:108A6600807D007C0012A29E783C12A66978BC121A
:108A7600A65D12A5A07F3F7E807D007C0012A29A93
:108A860012A5A0783C12A65D12A5A078B412A65D28
:108A960012A4AC12A4AC784012A669785412A65D52
:108AA60012A73B783C12A66912A5A012A4AC787452
:108AB60012A6697F417E107D007C0012A5A078C0B9
:108AC60012A65D12A4AC12A5A07F407E807D007C1C
:108AD6000012A5A0784412A65D12A4AC12A5A07F30
:108AE600417E207D007C0012A29A12A5A078441235
:108AF600A65D12A4AC12A5A07F407E407D007C003E
:108B060012A5A0787412A65D12A4AC12A5A07F408F
:108B16007EA07D007C0012A29E12A29E12A29A1234
:108B2600A5A0785012A65D12A4AC12A5A07850128A
:108B3600A65D12A4AC12A5A07F3D7E2A7DAA7CABC1
:108B460012A4AC12A5A07F3F7E007D007C0012A27D
:108B56009A12A5A0783C12A65D12A5A0787012A65E
:108B66005D12A4AC12A5A0784012A65D12A524122F
:108B7600A5A0785012A65D12A4AC12A5A07850123A
:108B8600A65D12A4AC12A4AC12A5A0785412A65DE0
:0C8B960012A29A12A5A07F4A7E517DD247
:108BA2007CCB12A4AC12A61278AC12A6697F407ECE
:108BB200007D007C0012A5A0787412A65D12A4AC00
:108BC20012A5A07F3F7E807D007C0012A29E12A58E
:108BD200A0784412A65D12A29E12A5A0785012A6F9
:108BE2005D12A4AC12A5A0785012A65D12A4AC121C
:108BF200A5A0785012A65D12A4AC12A5A07F3E7E5D
:108C02002A7DAA7CAB12A4AC12A5A0785012A65D54
:108C120012A29A12A5A0785812A65D12A52412A536
:108C2200A07F4A7E517DD27CCB12A4AC12A6121236
:108C3200A5A0AF3AEF3395E0FEFDFC12A5A07F4060
:108C42007E7E7D057C0012A88412A5A07F607E75C1
:108C52007D587CFF12A85D12A85D78B012A66978D3
:108C6200AC751B64128C898F1C78B0751B67128CD3
:108C720089E51C75F00AA42FFF249C50027F00781E
:108C8200D7E654802FF62275390012A65D12A5A0F0
:108C92007F0A7E007D007C0012A930A81BE513F636
:108CA20008E512F608E511F6335004EFF404FF224A
:108CB200C23D78647BAC1286A3D23D78677BB0124A
:108CC20086A31290BE7F007EE47D577C0012A5A091
:108CD20078AC12A65D12A85D12A5A07F007E537D1E
:0E8CE200077C0012A93012A5BF85133B7F80CE
:108CF0007ECB7DA47C0012A5A078B012A65D12A840
:108D00005D12A5A07F407E7E7D057C0012A93012F9
:108D1000A5BFE513F56F04F53A85126E85116D85D3
:108D2000106C7F407E7E7D057C0012A5A0786C12C1
:108D3000A65D12A88412A5A07F607E0C7DA27C0097
:108D400012A5A078B012A65D12A85D12A870786C6A
:108D500012A66978AC12A65DEC12A5D712A5A07F69
:108D6000347E9C7D2B7C5F12A4AC785412A66912D1
:108D7000A6ED785012A669786C12A65DEC12A5D704
:108D800012A5A07F347E9C7D2B7C5F12A4AC12A523
:108D9000A0785012A65D12A4AC784012A6697F405C
:108DA0007E007D007C0012A5A0785412A65D12A45E
:108DB000AC12A70312A5A07F3D7EC07D007C0012EF
:108DC000A5A078BC12A65D12A4AC12A5A07F3E7E21
:108DD000C07D007C0012A29E12A5A078BC12A65DE8
:108DE00012A4AC12A4AC12A5A07F3D7E407D007CF5
:108DF0000012A5A078BC12A65D12A4AC12A5A07F9B
:108E00003E7E807D007C0012A29E12A5A078BC123E
:108E1000A65D12A4AC12A5A07F3F7E807D007C00E1
:108E200012A29A12A5A0785412A65D12A4AC12A2A6
:108E30009A12A5A07F407E807D007C0012A5A078BC
:108E40005412A65D12A4AC12A70312A5A07F3D7E0A
:108E5000707D007C0012A5A078BC12A65D12A4ACA7
:108E600012A5A078BC12A65D12A4AC12A4AC12A2EA
:108E70009E12A5A078B412A65D12A4AC785812A6D2
:108E800069785412A65D12A703783C12A66978543B
:108E900012A65D12A73B785412A669783C12A65D13
:108EA00012A5A012A4AC12A5A078BC12A65D12A4B3
:108EB000AC783C12A6697F3E7EC07D007C0012A586
:108EC000A0783C12A65D12A4AC12A5A07F3F7E0044
:108ED0007D007C0012A29E12A5A0783C12A65D1215
:108EE000A4AC12A5A07F3F7E807D007C0012A29ED4
:108EF00012A5A078B412A65D12A4AC787012A6696F
:108F0000785012A65D12A5A012A4AC12A5A078C03C
:108F100012A65D12A4AC784412A669785412A65D1C
:108F200012A5A012A4AC787412A669784012A65DAE
:108F300012A5A012A4AC783C12A6697F407E807D69
:108F4000007C0012A5A0784412A65D12A4AC12A564
:108F5000A07F417E107D007C0012A29E12A5A07809
:108F60004412A65D12A4AC12A5A0787412A65D12DC
:108F7000A5A07F407EA07D007C0012A29A12A29E36
:108F800012A5A0783C12A65D12A4AC12A5A07F3D4C
:108F90007E2A7DAA7CAB12A4AC12A5A07F3F7E00E6
:108FA0007D007C0012A29E12A5A0785412A65D122C
:108FB000A5A0787012A65D12A4AC12A5A0783C12F0
:108FC000A65D12A4AC12A4AC12A5A0785812A65D9E
:108FD00012A29E12A5A07F3F7E7F7DE57CC912A4D0
:018FE000ACE4
:108FE10012A5A07F4B7E187D967C8012A29E12A6B0
:108FF1001212A5A07FE87E037D007C0012A9301229
:10900100A5BF78C8A61208A61308A60608A6077861
:109011007412A65D12A5A07F3F7E807D007C0012A8
:10902100A29A12A5A0784412A65D12A29E12A5A032
:109031007F3E7E2A7DAA7CAB12A4AC12A5A078400B
:1090410012A65D12A4AC12A5A0783C12A65D12A4D2
:10905100AC12A5A0784012A65D12A29E12A5A07F17
:109061003F7E7F7DE57CC912A5A0787012A65D12B6
:10907100A4AC12A4AC12A5A07F487EF47D247C0090
:1090810012A29E12A61212A5A07FE87E037D007C8B
:109091000012A93012A5BF78C4A61208A61308A60B
:1090A1000608A607223F3F4344454647484A4B4CE2
:1090B1004D4E5051525354555657583F3FE4F53990
:1090C100F5A79090D2791078B4E493F6A308D9F972
:1090D1002232A5C24A4A19DC3A885CDB3BFFD6DC66
:0190E1003B53
:10A22E00D2D58002C2D575A70490040078107F0B9A
:10A23E0012A25A78267F0512A25A783C7F2212A2C9
:10A24E005A786A7F0F12A25A75A7002230D506E6F9
:10A25E00F008DFFB22E0F608DFFB22D2D58002C237
:10A26E00D575A7049006FA78737F0612A25A75A7C1
:10A27E000022DA0CD902800BD906303701B3500513
:10A28E0002A40D923702A3F9D9F680F9D2368002D4
:10A29E00C23612A43E303606C86002B237C89236B5
:10A2AE00DAD0D9E4B8000A12A485A236923702A3F6
:10A2BE00E260FBB51300400F12A485A23692F7A2FE
:10A2CE00379236A2F79237C398F40424E740DF247E
:10A2DE0019AD29AC28AB277A00C394084008CDCC21
:10A2EE00CBCAE4CD80F424086010F9C3ED13FDEC65
:10A2FE0013FCEB13FBEA13FAD9F1A236303701B394
:10A30E0040308A17E5102BF518E5113CF519E512CA
:10A31E003DF51A501A13F51AE51913F519E5181328
:10A32E00F518E51713F5170513E51370020514025A
:03A33E00A398E4FD
:10A34100C39AF517E5109BF518E5119CF519E5126F
:10A351009DF51A500DB237C378177F04E496F608BD
:10A36100DFFA7A047019E513C39408F51350021546
:10A3710014E4C517C518C519F51ADAE802A439207D
:10A38100E7BAE5137002151415137817C37F04E6B5
:10A3910033F608DFFA80E8E51A20E7137817C37F60
:10A3A10004E633F608DFFAE513700215141513E518
:10A3B100173378187F03E63400F6500E08DFF7757F
:10A3C1001A800513E51370020514E51420E7547093
:10A3D10027E513604E046020851A1285191185182E
:10A3E100105326F0AC10AD11A237E51313FFE5129F
:10A3F10092E7FEA81302A5BFE4F512F511F510F5D9
:10A40100147513FF5326F043260580D8E5FFF51296
:10A41100F511F510751400F513D2375326F04326C4
:10A421000980C15326F0432603E4F512F511F51016
:10A43100F514F513C23780AC5326F080EC79017A1C
:10A44100018512F0E513A2F7339237751400F51365
:10A451006002D2F785F012A813B8FF0809E512C20D
:01A46100E713
:10A462006001098C278D288EF0A2F7EF3304700A61
:10A472000AC2F705F00AD5F0011A146002D2F78574
:10A48200F02922C88813C512C529C512C511C528CD
:10A49200C511C510C527C51022DA03B8000302A4EE
:10A4A2000DD9028002D9F702A3F912A43E30370176
:10A4B200B392377004D9E78005DADEB8000302A44C
:10A4C20039D9E2C3947E500215142513F5135002B4
:10A4D20005147815760008B81BFA78277915E6086E
:10A4E200FAE8FC78108AF0E608A427F709E5F037C5
:10A4F200F7500989F00907E760FBA9F0B813E619DC
:10A5020019ECF8B82AD802A39802A424B8FFFA02D8
:10A51200A40DD9FB02A3F9DAF6B800F002A43912AD
:10A52200A67512A43E303701B392377007D9E3B84B
:10A5320000E280DBDAE1B8000280E1D9D5C8C39835
:10A5420050021514247F50020514F513781A760070
:10A552007A1A7B80C3E5109527E5119528E51295B7
:10A56200294016C3E5109527F510E5119528F51138
:09A57200E5129529F512E64BF6FD
:10A57B00DA0302A398EB03FB30E703187600C3E57D
:10A58B001033F510E51133F511E51233F51240CA0E
:10A59B0030E7DD80B6E53905396010D0F0D0E0C08A
:10A5AB0010C011C012C013C0E0C0F08F138E128DFB
:10A5BB00118C1022E539146010D0F0D0E0D013D0FC
:10A5CB0012D011D010C0E0C0F01539227920800CC8
:10A5DB007910800479087D007E007F003392D5507E
:10A5EB000312A64FEC33400FEF33FFEE33FEED3388
:10A5FB00FDEC33FCD9EE22EECCF5F0747E29A2D51E
:10A60B0013FF92F7AEF022EF8EF0A2F7D2F7339250
:10A61B00D5C3947F5006E4FFFEFDFC22942040043A
:10A62B0074FF80F304CCFEE4FFFAE5F0CC6012C3B8
:10A63B00CC13CCCD13CDCE13CECF13CF0450EEDA3B
:10A64B00EC30D5D7C3E49FFFE49EFEE49DFDE49C74
:03A65B00FC22E6F8
:10A65E00FC08E6FD08E6FE08E6FF22ECF608EDF63D
:10A66E0008EEF608EFF622CFC513CFCEC512CECD2B
:10A67E00C511CDCCC510CC22E4F513F512F511F5AC
:10A68E001022E493FCA3E493FDA3E493FEA3E493CE
:10A69E00FFA322C0E012A5A012A4AC12A6D412A64B
:10A6AE0090D0E0C0E012A5A012A6CB12A4AC12A5C9
:10A6BE00A012A69012A29ED0E0D5E0E722AC48AD43
:10A6CE0049AE4AAF4B228C488D498E4A8F4B22742D
:10A6DE00FF7809FFFEFDFCE52654F048F526221210
:10A6EE00A79404A2E1927F1420E01590A81574049B
:10A6FE0012A6A1802912A79430E102B27F20E0EBCE
:10A70E008C4C8D4D8E4E8F4F90A829740412A6A19D
:10A71E0012A5A0AC4CAD4DAE4EAF4F12A4AC307FD7
:10A72E0004EF6480FFEE33EF337001FF2212A79423
:10A73E00C0E08C4C8D4D8E4E8F4F90A84D740312F1
:10A74E00A6A112A5A0AC4CAD4DAE4EAF4F12A4AC0F
:01A75E00EC0E
:10A75F00C54CFCEDC54DFDEEC54EFEEFC54FFF9050
:10A76F00A83D740312A6A1D08212A5A0AC4CAD4D8A
:10A77F00AE4EAF4FE58230E00712A524B27F809D29
:10A78F0012A5218098EE33EF3324605007D0E0D02C
:10A79F00E002A6DDEFA2E7547F927FFF12A5A07C17
:10A7AF00837DF97E227F3E12A4ACEE33EF332481FA
:10A7BF00501012A5A012A61212A5D7EFB2E7FF12E2
:10A7CF00A29EEE33EF33602A2403F8C313FFEE92F9
:10A7DF00E7FEE82481E4501A12A5A012A612EF0496
:10A7EF00C2E0FCF58212A5DFEFB2E7FF12A29EE5F1
:10A7FF008203FAEE33EF33600B148FF0A2F713FFDF
:10A80F00EE92E7FEEA2283FA703AE4E9AABCF8E096
:10A81F00813EE6E99DBF0000803F1A3C28396669FA
:10A82F0099BBE335A33DE75D25BFDB0FC93FCCDB0C
:10A83F008D41EE3649C43F91C9453DF8B0C5000082
:10A84F00803F34F517C373FA2F45DDFD0AC6EF2598
:10A85F0013FFEE3512FEED3511FDEC3510FC02A5A0
:10A86F00BFC3EF9513FFEE9512FEED9511FDEC951D
:10A87F0010FC02A5BFEFF88513F0A4FFE513C5F098
:0AA88F00CEF9A42EFEE435F0CDFA58
:10A8990088F0E512A42EFEED35F0FDE433CC8513E6
:10A8A900F0A42CFCE5128AF0A42CFCE51189F0A493
:10A8B9002CFCE51088F0A42CFC89F0E512A42DFDF0
:10A8C900EC35F0FCE51188F0A42DFDEC35F0FC8A9F
:10A8D900F0E513A42DFDEC35F0FC02A5BFE4CCF89E
:10A8E900E4CDF9E4CEFAE4CFFB75F020C3E51333E8
:10A8F900F513E51233F512E51133F511E51033F5CA
:10A9090010EF33FFEE33FEED33FDEC33FCEF9BEE3E
:10A919009AED99EC98400CFCEF9BFFEE9AFEED99AD
:10A92900FD0513D5F0C622C2D5EC30E705B2D51224
:10A93900A64FE51030E70DB2D512A95312A8E612B9
:10A94900A64F800312A8E630D515C3E49513F51375
:10A95900E49512F512E49511F511E49510F510221C
:109A1100E57124885002D219125F428E4712C43276
:109A21001286011262EB305E0F126289127D2612DC
:109A310061C712B331123D0E1234541242D710369F
:109A410029201F1C301219E4129B97129BAC129C07
:109A5100AE129CD0305103029D5A12A02B20510905
:109A6100C251E4F552F545F5442275A70075830707
:109A7100E559C454F0F582E0F538A3E0F518A3A345
:109A8100A3E0F51E74FF129B97125F428E1C8F1B81
:109A91007510DF751100E51164B47006129B6275D3
:109AA1001110129B2F4028AE1CAF1B125FC8203231
:109AB1001EAC03AB027A0C125BF1ED701275A700BC
:109AC100758304851182ECF00583E510F00511D54D
:109AD10010C4129B6275C70375C6E075A704900593
:109AE100007F04129B1DDFFB75A7001225DC1262AB
:109AF10089E4F5A7F8F559758307E8C4F582E065AF
:109B0100387011A3E06518700BA3A3A3E0651E7064
:109B11000388592208C3E5589850DC22E0F5BCE0DF
:109B2100F5BDE0F5BEE0F5BF1248EB05C622E51034
:109B310075F004A4F5C685F0C775B901E5BC3340DD
:0B9B41001F05C605C675B90185BE648E
:109B4C0085BF6505C675B90185BC6685BD6785BED3
:109B5C006885BF69C322E51124FE502E75A7007FCE
:109B6C0010AE111E7583048E82E0FD1582E0CDB51A
:109B7C0005005012F00582CDF00583E0FD1582E062
:109B8C00CDF00582CDF0DEDCDFD72275A754900432
:109B9C000005A79005007FB4F0F0DFFC75A700224C
:109BAC0012B17DC2517B077AFFE4FFF5A790040048
:109BBC00129C92ED244C4035EC603075A7008D82E0
:109BCC0005A7129C587583058D82E02410401CF06B
:109BDC0005A7E02CF0500505A7E004F0BA000CBB7B
:109BEC000009D251EF24DC50027F23DFC3EA600569
:109BFC00129C0B8006EB6003129C4375A70022306D
:109C0C00E0047553082230E1047553182230E20445
:109C1C007553282230E3047553382230E40475530D
:109C2C00482230E5047553582230E60475536822F7
:109C3C0030E7037553782230E0047553882230E105
:109C4C00047553982230E2037553AA22ED54F0C4E4
:109C5C002323909C62735302FE225302FD22530273
:069C6C00FB225302F72267
:109C72005302EF225302DF225302BF2253027F22FA
:109C82005303FE225303FD225303FB225303FB2201
:109C920012B08F12AF1CE4F5F7C2B2C2B2ADF7F543
:109CA200F7C2B2C2B2ACF7D2B2C22022900500789B
:109CB200B4E06015FD54F0C4CD7C00540FFE158352
:109CC200E0FF125CEFEFF005830582D8E422758392
:109CD2000478FF088882E060FAF5D38812E512243E
:109CE2004C50012285D3D288D4881279FF0512E51F
:109CF2001260F00908E875F0B484A8F08882E06088
:109D0200ECF5D3B9000280D5B9230050D0C395D267
:109D120092D15002F40409FEE4FFFCAD01125CFC96
:109D22007401FA25D475F0B484A8F0AC06AB07121E
:109D32005BE3EB30E7010CE5D22C30D1029C9C882E
:109D420082F00AEAB501DCE512244C50012285D3E7
:109D5200D28512D4A8128093900400129E198C0608
:109D62008B05129E19E4FFF512F5118C148B13C3A7
:0E9D7200ED9BF9EE9CFA4012E51199E5129A6C
:109D8000500A8C148B138A1289118F528F82E0F93A
:109D9000C3ED99FDEE9400FEE582245A5002244C56
:109DA00075F0B48485F082E0FA2DFDEE3400FEEB10
:109DB0009AFBEC9400FCE92BFBEC3400FC0FBFB4E5
:109DC000B0E55224D3400224B4F552C3E51333FB6B
:109DD000E51433FCE511FE2BFBE512FF3CFC125DA4
:109DE00051E9F8909E2B93F511FDEBF513FFECF57F
:109DF00014FE7C00125CEF8F44E8909F2B93FAAB2B
:109E000013AC14125C1AAF03AE04AD117C00125CEB
:109E1000EFEF7002F552F545227C007B007F5AE09F
:109E20002BFBEC3400FC0582DFF522B4B4B4B4B4EF
:109E3000B4B4B4B4B4B4B4B4B4B4B4B4B4B3B3B3E5
:109E4000B3B3B3B3B3B3B3B3B3B3B2B2B2B2B2B2E8
:109E5000B2B2B2B1B1B1B1B1B1B1B0B0B0B0B0B0F5
:109E6000B0AFAFAFAFAFAEAEAEAEAEAEADADADAD0F
:109E7000ADACACACACACABABABABAAAAAAAAA9A933
:109E8000A9A9A9A8A8A8A8A7A7A7A7A6A6A6A5A55F
:109E9000A5A5A4A4A4A4A3A3A3A2A2A2A2A1A1A194
:109EA000A0A0A0A09F9F9F9E9E9E9D9D9D9D9C9CCF
:109EB0009C9B9B9B9A9A9A9999999998989897970D
:109EC000979696969595959494949393939292924F
:109ED000919191919090908F8F8F8E8E8E8D8D8D90
:109EE0008C8C8C8B8B8B8A8A8A89898988888887D5
:109EF000878786868685858584848483838382821A
:109F0000828181818080807F7F7F7E7E7E7E7D7D5D
:109F10007D7C7C7C7B7B7B7A7A7A7979797878789E
:109F20007777777676767575757474000203050613
:109F300008090B0C0E101113141617191A1C1D1FEB
:109F40002122242527282A2B2D2E30313334363751
:109F5000393A3C3D3F404243454648494B4C4E4FC1
:109F6000505253555658595A5C5D5F606163646640
:109F700067686A6B6C6E6F707273747677787A7BD1
:109F80007C7E7F80818384858688898A8B8D8E8F75
:109F90009091929495969798999B9C9D9E9FA0A135
:109FA000A2A4A5A6A7A8A9AAABACADAEAFB0B1B20A
:109FB000B3B4B5B6B7B8B9BABBBCBDBEBFC0C0C1FB
:109FC000C2C3C4C5C6C7C7C8C9CACBCCCCCDCECF07
:109FD000D0D0D1D2D3D4D4D5D6D7D7D8D9DADADB2A
:109FE000DCDCDDDEDEDFE0E0E1E2E2E3E4E4E5E567
:109FF000E6E7E7E8E8E9EAEAEBEBECECEDEEEEEFBA
:10A00000EFF0F0F1F1F2F2F3F3F4F4F4F5F5F6F623
:10A01000F7F7F8F8F8F9F9FAFAFAFBFBFBFCFCFDA4
:10A02000FDFDFEFEFEFEFFFFFFFFFFC251E4F54413
:10A03000F814FB900400A9007C0FC2D112A146E8DD
:10A040002405F8B8B4F08B13E5122403FA244C501D
:10A0500001FABBFF012275112C8A1912A17D8F16FE
:10A06000203D12AA1975112312A17D8F15751600B6
:10A07000303DE2801175112312A125751500303D88
:02A0800005E8F1
:10A082002F13F51575111212A125751400303D0517
:10A09200E82F13F514EA2404F552244C5002F55229
:10A0A200E4F51AF51BF51CE516600AFB7A00AF13FE
:10A0B2007EFF12A0EBE515600AFB7A4FAF137EFF1D
:10A0C20012A0EBE516600DFB7A00E5146006FF7E38
:10A0D200CF12A0EBAE1CAF1B7C00AD1A125CEF8F4F
:10A0E20045EF2513F544D25122EFF5F0A4FCADF073
:10A0F200EBF5F0A49CFCE5F09DFDEB8AF0A4FAAB35
:10A10200F0EF8EF0A49AF8E5F09BF9E833F8E93322
:10A11200F97B00125D95051AE51B2BF51BE4351C36
:10A12200F51C22EA2511F9244C5001F9C2D112A1E1
:10A1320044303D428F00C3EA9511F9500324B4F92B
:10A14200D2D17C09E4FDFEFF8982E060062FFFE4A4
:10A152003EFE0D09B9B4027900DCEDED20D118F50F
:10A162001E24FE923D500F125CFCEFB50300500618
:0EA17200851E1FFB881222F51D80E612A12516
:10A18000203D43740212A21C12A125203D38740404
:10A1900012A22412A125203D2D740612A21C12A188
:10A1A00025203D22740812A22412A125203D1774F7
:10A1B0000A12A21C12A125203D0C740C12A224121A
:10A1C000A125203D0122C3E89F605088148F158A85
:10A1D0001640081ABAFF0A7AB380060ABAB4027A9D
:10A1E0000012A125303D34C3E89FF9602EC3E51469
:10A1F0009515FB6930E7D4E930E703F404F9EB3057
:10A20000E702F404C3995002AA16E5142515C82FD5
:10A2100028FFE4FC33FE7D04125CEF222AFA244C72
:0EA220005001FA22C3CA9AFA500324B4FA225B
:10AEEA00C2B212D07DD2B275F83022C2B2F5F7C220
:10AEFA00B2C2B2D2B222D220C2B2F5F7C2B2C2B242
:10AF0A00856CF7C2B2C2B2856BF7C2B2C2B2856AA9
:10AF1A00F722D220C2B275F703C2B2C2B2856FF766
:10AF2A00C2B2C2B2856EF7C2B2C2B2856DF722D280
:10AF3A002012AF6D740612AEF5740212AF008FF7CD
:10AF4A00C2B2C2B2D2B2C22022D21412099B125A7F
:10AF5A00F01248EBD22012AF6D740612AEF574C728
:10AF6A0012AEF512AF7340FB22C2B275F705C2B238
:10AF7A00C2B2C2B2C2B275F705C2B2C2B2C2B2C2DC
:10AF8A00B2E5F7D2B2A2E02212099B85BF6C85BE58
:10AF9A006B756A00E56B7019E56A7015D22012AFFD
:10AFAA006D740612AEF574D812AF00D2B2D21F0574
:10AFBA004DC22022E54B0475F03C8485F04B12B259
:10AFCA00A9852E72E55F030354C0F8E55E543F2855
:10AFDA00F57C3055012212B01912AF7340F7E54CD7
:10AFEA0060F312AF6D12B03012AFFA80F112AF6D8A
:10AFFA00C21FD220740612AEF5740212AF00787026
:10B00A0086F708B880FAD2B2C22012B04D8085788D
:10B01A007075A704758304E54CC4F5827F10E6F0C9
:04B02A00DFFC054CF6
:10B02E008019787075A704758304154CE54C30E7CC
:10B03E0001E4C4F5827F10E0F6DFFC75A7002274F0
:10B04E0010256A54F0F56AE4356BF56BE4356C54F3
:10B05E000FF56C22E54B75F010A4256A54F0F56AD5
:10B06E00E5F080E4E56A24F054F0F56AE56B34FF10
:10B07E00F56BE56C34FF80D7E56A24FF80ECC38066
:10B08E00EBE56D24F054F0F56DE56E34FFF56EE5ED
:10B09E006F34FF540FF56F2275A7047583048F82EA
:10B0AE007870E6F008B880FA75A7002275A70490AC
:10B0BE0004B47F20E4F0DFFD80EE12B12412B15013
:10B0CE00C22DC254C255E57F7002D255147002D201
:10B0DE0054E54A30E00122B4061E20540F12B0721D
:10B0EE0012B1F412B28812B2C002B3D01279F37E4A
:10B0FE000412D075754A012220550F12B04D12B2AE
:10B10E006712B2A912B1CD02B3A31279F37E041263
:10B11E00D075754A0522740312AF007870E4F5F706
:10B12E00C2B2C2B2A6F708B880F3D2B2C22022745D
:10B13E000312AF00E4F5F7C2B2C2B2E5F7D2B2C263
:10B14E002022E575F8541F30E40244E0F57585724F
:07B15E002EA2779226E57C8A
:10B16500543F30E50244C0F55EE57C54C02323F529
:10B175005FE57F1414F55122856C6F856B6E856ACA
:10B185006D22856F6C856E6B856D6A22E4FEFF749A
:10B195000775A704F5838E8274FFF0DFFD75A700A0
:10B1A5002274067E007FB012B196E4F55AF55B2253
:10B1B50075A704758306E55A600A75F00A84E5F0FB
:10B1C5007002740AC4F58222307720E55A240240C1
:10B1D50002055A12B1B5E55AF0E573F0E574F0E5EC
:10B1E50075F0E576F0E577F0E578F075A7002230A3
:10B1F50077F912B1B57F1074FFF0DFFDE55A24F53C
:10B20500500312B21F155AE55AB4FF02055AC3E599
:10B215005A955B50D6755B0080D112B17D7F0A05CA
:10B225006D056D12AF1CE4F5F7C2B2C2B2E5F7D2F7
:10B23500B2C22030E704DF02800512B08F80E0053E
:10B245006D12AF1C12B1B5E55A24F6F07F06E4F590
:10B25500F7C2B2C2B2E5F7F0DFF4D2B2C22075A7E9
:10B265000022053FE53FB43C17753F00053EE53E2E
:10B27500B43C0D753E00053DE53DB41803753D0034
:10B285000245AD153FE53FB4FF17753F3B153EE55C
:01B295003E7A
:10B29600B4FF0D753E3B153DE53DB4FF03753D1707
:10B2A6000245AD0542E542B43C0F7542000541E555
:10B2B60041B43C057541000540221542E542B4FF04
:10B2C6000F75423B1541E541B4FF0575413B1540FD
:10B2D60022AC40AB41A842EC75F03CA42BFBE43514
:10B2E600F0FC7A3C125BE3EB28FBE43CFC22AC3D31
:10B2F600AB3EA83F80E178AE8604AB3EE53FC31384
:10B30600F88011120991ACBF53041FE5BE75F00514
:10B31600A4FB7800EC75F03CA42BFBE435F0FC7A3A
:10B326001E125BE3EB28FBE43CFC2212B309AE04DD
:10B33600AD0312B2FC8C148B1312096EE5BFFF2409
:10B34600F650027F01E5BE75F096A4AAF0F9C3EDAA
:10B356009513FBEE9514FC924E4B701120110E3096
:10B36600480B75364B3003037536FFD22E304E022E
:10B37600DF1F7A02125BE375A7009004EEECF0A3E0
:10B38600EBF0C3E5BF9F04BF0102D2E79005CBF007
:10B3960022ED29FDEE3AFE80B520740122C3E57048
:03B3A6009557FFB9
:10B3A90024FD5021EF24EB400A78BD06B60016189B
:10B3B900068012EF2402400DEF2414500878BB06D2
:10B3C900B600021806802BC3E5709557FF24FD507F
:10B3D90021EF24EB400A78BB16B6FF161816801227
:10B3E900EF2402400DEF2414500878BD16B6FF0271
:06B3F900181685705722B2
:10D0620012D06B12D06B12D06B7E0480067E0280CF
:10D07200027E017F0080087F6480027F017E00EFD4
:10D082004E6012E4FD0D1D0DEDC394AD40F7EF1F90
:10D0920070ED1E80EA22753500C200C201C2022272
:10D18800F5D8D2DCE5F520E7FBE5DA540FFEAFD998
:04D1980075D8002224
:10CDBE007F767E069090F7126C09740412D1887CEF
:10CDCE00007D52125CEFEFF875F00A84C0F07F76AA
:10CDDE007E2312C70C7E29742E12C71F7E2ED0E022
:10CDEE0012C70C7E35745612C71F7F6B7E1190CE04
:10CDFE002712C74DE824E04001220423F824E7500F
:10CE0E0002781812CE17D8FB227F6CE82411FE7917
:10CE1E000512D0E10E0FD9F922071DFFFFFFE080AA
:10CE2E00000020C0000038E0000008F0000038F8D4
:07CE3E00000020FFFFFFE0F0
:10CEC30012CEEB30E6022409540F75F00AA4F515CF
:10CED30012CEEB30E6022409540F25152212CEEBB5
:10CEE300540F2275F000800875F044800375F00735
:10CEF300E4206D09D5E0FAD5F0F7D24C229247C26F
:10CF0300ACE54F623885504FA26E926D859950C241
:10CF13006FD2ACC24CA2472212CF25C4FA12CF253E
:10CF23002A2212CEEB20E603540F225407240922AF
:10CD2C00E612CD3318E608FAC412CD39EA540F4492
:10CD3C0030F924C6E950112407800D75F00A84C01F
:10CD4C00F012CD52D0E0443030530975F00085E03C
:10CD5C00E0D5F0FA3099FDC299F599623822E538A0
:10CD6C0080F2E53812CD33800812CD54E53812CD5F
:10CD7C0054740D12CD54740A80CE744012CD547478
:10CD8C004080C5742C80C1742E80BD12CDAFE912C9
:10CD9C00CD60800312CDAFE812CD60E53812CD60C6
:10CDAC00024355124355800312436D74407538008D
:02CDBC0080965F
:10D1AE0085A0835383FE438380858384F07584003A
:01D1BE00224E
:10CBDA0074A212D1AE74A112D1AE74A612D1AE74DF
:10CBEA00A412D1AE74C012D1AE742512D1AE12CC39
:10CBFA006A75C70375C6FC75B90112A9697408126A
:10CC0A00D188EE75F020A4FEEF54F80303032E2416
:10CC1A0092C313FE24EA50027E16EE90CC5393255B
:10CC2A00BCFE24E6501F24E8401B748112D1AEEEEC
:10CC3A0012D1AE12CC77744012D1AE742F12D1AE8B
:10CC4A0074AF02D1AE7E2680E1F7F7F8F8F9FAFB65
:10CC5A00FCFDFEFF000000000101020202030303C3
:10CC6A00A8BCA9BDAABEABBFACC7ADC62288BC8949
:0ACC7A00BD8ABE8BBF8CC78DC62299
:10CFDC00D21AC006C007C0E075A7019000007EB74A
:10CFEC0075A700EE12D1AE741012D1AE740412D12A
:10CFFC00AE85A08343838185838475A7517F80E0B0
:10D00C00F0DFFC1EBEAFD9E4F5A7F584D0E0D00765
:05D01C00D006C21A223B
:10D19C0075A711900000E4C583F0C58330E2F8F563
:02D1AC00A722B8
:10D0E100EF20E723EE20E71F20E61C05A7C4540329
:10D0F100F583EE5408C42FF582EE5407240983F515
:10D10100F0E045F0F005A72280402010080402015C
:10D11100EF20E723EE20E71F20E61C05A7C45403F8
:10D12100F583EE5408C42FF582EE5407240983F5E4
:10D13100F0E055F0F005A7227FBFDFEFF7FBFDFE22
:10C6CC00FDA42582F582E5F03583F583ED22906893
:10C6DC00577A0475F00512C6CC7D0580607A05800A
:10C6EC00027A04547FC0E0C083C082C394205001FE
:10C6FC00E490680712C6DF80309069657A05800582
:10C70C00906A227A0675F00712C6CC7D07802E7AC5
:10C71C000580027A06547FC0E0C083C082C3942097
:10C72C005001E49069B212C711D082D083D0E022BC
:10C73C0090678575F00A12C6CC7D0A7A07C2D18043
:10C74C0002D2D1C0A7C082C083C007C006C0E030EF
:10C75C00D10975A704E493FDE493FAEEFB75A704E5
:10C76C00EBFEEAFC7901D9067908E493F5D4E5D41B
:10C77C0023F5D420E01612D1110EDCEA0FDDE1D046
:10C78C00E0D006D007D083D082D0A72212D0E1808F
:10C79C00E89066C575F00E12C6CC7D0E7A0812C7ED
:10C7AC004990676D75F00212C6CCE493FDE4A39337
:10C7BC00FACE2408CE7C0812C7CA7C06AD02ED2343
:10C7CC00FD20E00712D1110FDCF42212D0E180F72A
:10C5B700F5D2C2D58036F5D2D2D58030F5D224F661
:10C5C70050090E0E24A650030E0E0EE5D2F5D275B5
:10C5D700F0648485F0D3C2D57009D2D5742012C710
:10C5E7001F800312C70CCE2406CEE5D375F00A844C
:10C5F70085F0D3700A30D507742012C71F80031245
:10C60700C70CCE2406CEE5D312C70CE5D222F5D24D
:10C6170075F0648485F0D3C2D58022F5D2C2D58067
:10C6270025F5D2D2D5801FF5D275F0648485F0D375
:10C63700C2D57009D2D5742012C71F800312C7054F
:10C64700CE2405CEE5D375F00A8485F0D3700A3081
:10C65700D507742012C71F800312C705CE2405CE45
:10C66700E5D312C705E5D222F5D2C2D58035F5D27A
:10C67700D2D5802F30E70DF404C0E0742D12C6ED3B
:10C687000E0ED0E0F5D275F0648485F0D3C2D57074
:10C6970009D2D5742012C6ED800312C6DACE24045F
:10C6A700CEE5D375F00A8485F0D3700A30D50774C8
:10C6B7002012C6ED800312C6DACE2404CEE5D312CB
:05C6C700C6DAE5D222F5
:106BF7007E00800E7405FEF51EE4FFF51DF51F20CF
:106C07003C3375A700E493700122A3B40204051D69
:106C17008003B4010A051FEF2409FFAE1E80E612A8
:106C2700C71F7D06B440027D03B421027D02EE2D0D
:106C3700FE80D27E0075A700E493700122A3B40200
:106C470004051D8003B4010F051FEF2407FFAE1EC7
:106C570080E612C6E98008B45B0050F612C6ED0E56
:106C6700B4210280D30EB4400280CDB42C0280C878
:106C77000E0EB45F0280C1B45B0040BC0E0E80B83C
:106C8700E60812C71FEE2406FED513F4229090FCE7
:106C9700307409909100307303909105026C097567
:106CA700F019D5E0FDD5F0FA12431B12CD86744FCB
:106CB70012CDB9744B12CD75C322C250126D051295
:106CC700431BD2AC12CEE6304C1212CEE6304C0C3F
:106CD70012CEE6304C06D250C2ACD322B440E512F5
:106CE700CEEBB4400312CEEBB44FED12CEEBB44B68
:106CF700E712CEEB12CEEB12CEEBC2ACC32230536F
:106D07000975F008D5E0FDD5F0FA227F0575F01971
:106D1700D5E0FDD5F0FA12431B12CD86745712CD7C
:106D2700B9745012CD54748112CD54E56312CD5409
:076D3700E56212CD5478D093
:106D3E00E612CD5408B8D7F8E6F8795F30E7027955
:106D4E002FE912CD5412CD5412CD5412CD54745885
:106D5E0012CD54744312CD54E412CD54E8C2E775EB
:106D6E00F00A84C425F012CD547864E612CD54088E
:106D7E00B869F8E612CD75126CC1400122DF0280AF
:106D8E000A20508B75F0008080D250C2ACD32212F4
:106D9E006D05C25012431BD2AC2002EF12CEE6207C
:106DAE004CE7B440F412CEEBB4400312CEEBB45722
:106DBE00DAF53812CEEBB450D212CEEB12CEEBF592
:106DCE006312CEEBF56278D012CEEBF924A050030D
:106DDE0053015FE924E04002795FA60108B8D8E8C4
:106DEE00780612CEEBD8FB12CEEBFC53040FC45434
:106DFE000F75F00AA42CFC249C50027C0078D786D8
:106E0E0001E4B92F02D2E72CF6786412CEEBF60825
:106E1E00B86AF812CEEBE5386003026D9912CEEB2C
:106E2E0012CEEBC2ACC3229096EC80039093917F6E
:106E3E0020126C3A12CFDC02D073753400C26B1282
:106E4E006EFD12D07312726FE5166003126E600241
:106E5E0002571274D31218DF12CFDC10002010016B
:106E6E000280F81272DA50131218EA126E35100000
:106E7E000D10010280F812188C80D712705B22C29E
:036E8E006BD2279D
:106E910075480A1225D07534001273A9C26A122FDF
:106EA1001C106A0512024880ED120248127201128A
:106EB10073591273B51274D31218DF12CFDC10009C
:106EC1003810010280F81272DA501BE9651560185A
:106ED1001218EA126E3512D06B10001D10010280DB
:106EE100F812188C80C3D26B1273857516078559F9
:106EF10017122649753500809D02025712726F12D2
:106F01006F1F1273B57F19126F399097197E121284
:106F11006C3C7E23E51602C68B90981280EF786256
:106F2100E4126F3078D0745F126F3018E4F6227F6C
:106F310008F608DFFC227F7B7E007810742012C6E1
:106F4100EDCE2404FED8F5227F197E08126C3C7E1A
:106F510028909373305303909378026C3CC26B1268
:106F61006F1F126F69020257C2511273B5909711C8
:106F7100126F491218B212726F7F20126F0812CF6E
:106F8100DCE516700512D068803675A6FF30510316
:106F9100126CAF12431BD2AC200025306DFA126D7A
:106FA100A0400C1272DA401112705BD25180BB10FA
:106FB1005003126E3AC25180D1D251126E3580CA3D
:106FC100C2AC22D22775480A1225D0753400C26B93
:106FD1001273A9C26A122F1C106A0512024880EBB3
:106FE1001202481272011273591273B5126FF550E1
:106FF100DA02025790938C126F491218C412CFDC37
:04700100C3100013A5
:1070050010010510020E80F4126D12400122126E5D
:107015003A80DDD3C2AC22D227C26B75480A12254D
:10702500D07534001273A9C26A122F1C106A05129A
:10703500024880EDD26B12720112735912722975D2
:10704500B901E5BCB2E7F5BC1248EB7516078559E1
:107055001712264980CBD26B127385127240E51741
:1070650075F01084240AF54824E8500375480A127F
:1070750025DC85585922D22075320012B19175A7A9
:107085000490070075150012722975B901E5BC2039
:10709500E705E515F0801004600D6482600975BC94
:1070A500FF75B90575B9020515E515242050D8E514
:1070B5008224FE4003027156A882187F0075A7003E
:1070C5007583078882E0FE75F004A41271D4A9BC0B
:1070D500AABDABBEACBF1582E0FD75F004A412716C
:1070E500D4C3E995BC404C7052EA95BD4045704B00
:1070F500EB95BE403E7044EC95BF4037703DEE7554
:10710500F004A4041271D4A9BCAABDABBEACBFEDFA
:1071150075F004A4041271D4C3E995BC4015701B25
:10712500EA95BD400E7014EB95BE4007700DEC95C9
:09713500BF5008EEF00582EDF0F8
:10713E001582E5826009C3EF958250030270CA0F73
:10714E00C3E89F40030270C275A70490070075C77D
:10715E000375C6A8E0F5BCE0F5BDE0F5BEE0F5BFF1
:10716E0075B90575B90205C6E58224204006E5C647
:10717E00242050E00875C70375C68075B901E5BCBB
:10718E001271BEF5BCE5BD1271BEF5BDE5BE127144
:10719E00BEF5BEE5BF1271BEF5BF75B90205C6E5F7
:1071AE00C6245850D6E5320470FB75A700C22022C3
:1071BE00B4FF0122F975A704900700E58268600507
:1071CE00E06970F7E922F5C685F0C775B901E5BC2F
:1071DE00645F700375BC27E5BD645F700375BD27E2
:1071EE00E5BE645F700375BE27E5BF645F7003750F
:1071FE00BF272275C703E54875F004A42480F5C6A1
:10720E00E55975F00484A8F00825C6F5C675B901D0
:10721E00A9BCAABDABBEACBF861522E51524205075
:10722E00037515DFE51575F004A454FCF5C685F05D
:10723E00C722E51724204028E51775F00484A8F02E
:10724E000824A8F5C675C70375B901A9BCAABDABBC
:10725E00BEACBFA61589BC8ABD8BBE8CBF1248EBD7
:02726E0022E418
:10727000F516F51579FF12722975B901E5BCB4FF51
:10728000040516A9150515E515242050E989157979
:10729000FF75C70375C6A875B90109E5BC04601B75
:1072A00009E5BD04601509E5BE04600F09E5BF04EA
:1072B000600905C6E5C6242050DD09891722751628
:1072C0000075150112722975B901E5BC20E70205A8
:1072D000160515E515242050EB227900E975F00418
:1072E000A454FCF5C685F0C775B901E5BC20E730AC
:1072F00078D066702B08E5BD66702508E5BE66701F
:107300001F08E5BF66701905C675B90108E5BC66BA
:10731000700E08E5BD66700808E5BE667002D322EF
:1073200009E9242050B6C322127348127330A80111
:107330007F08E0F608DFFB22127348127340A801B1
:107340007F08E6F008DFFB2278D0796275A7047524
:107350008307EBC454F0F5822212722978D012739D
:1073600073E5BCF9C23C20E702D23C127373786229
:1073700012737375B901A6BC08A6BD08A6BE08A6FF
:07738000BF0805C622D22060
:1073870012722978D01273971273977862127397D3
:1073970086BC0886BD0886BE0886BF081248EB056E
:1073A700C62212628912D19C127B2902CFDC12D12C
:1073B7009C7F007E099096FE126C097F0A7E12E57B
:1073C700150412C5C37F1412BD8912188C7F277E3E
:1073D7000875130778D0126C87E6793E30E7027993
:1073E7002F7E34E912C71F7F3D7E0190982E126CC5
:1073F7003C20311B303003128621C23B12766512C6
:10740700741BD23B12766512742D1276AC807C12F7
:10741700B3FF80E6C23B7F447453201702744E7E4D
:107427000012C71F8017D23B7F4F74572017027473
:10743700457E0012C71F7E06E51E12C70C7E0CE5AF
:107447001D12C70C7E12E51C12C70C7E177464123E
:10745700C71F7E1CE51B12C70C7E22E51A12C70C3C
:107467007E28742E302602742712C71F7E2DE51939
:1074770012C70C7E33E51812C70C7E393026077405
:107487002C12C71B7E3BE53702C70C742D20170251
:10749700742B7F707E1512C71F1274B07E3A12C507
:1074A7006C7E01909859026C097E1BE51C12C70C73
:1074B7007E21E51B12C70C7E27E51A12C70C7E2D0D
:1074C700E51912C70C7E33E51802C70C1275511265
:1074D700757C1278531273B51278AB20171E100201
:0774E7001B1243E212BB9EE1
:1074EE001275391218977F347E2F126C941273EE28
:1074FE0012CFDC80E212188C203026203128C23BBD
:10750E001276651275917866127765D23B127665A2
:10751E001275A678691277651276AC12762002780B
:10752E00081286EA80F212B41480EDE57D75F01033
:10753E0084AAF075F00AA42A547FFA78D7E654800C
:10754E002AF6227F277E0879D08700C001D224B97F
:10755E00D002C224127932D001A70010230909EEFD
:10756E002406FEB9D7E32219EE24FAFE80DB7E3420
:10757E0079D7E7A2E792171278DF79D7E7A21792A9
:10758E00E7F722C224C23B751E007F447E001278AC
:10759E00EF801E1023ED802AD23BC2247F4F7E0047
:1075AE001278F7D2247E06E51E127924F51E1023DA
:1075BE00E7D2247E0CE51D127924F51D303BD41044
:1075CE0023E1D2247E12E51C127924F51C1023E14E
:1075DE007E1CE51B127924F51B1023E67E22E51A8C
:1075EE00127924F51A1023E87E2DE519127924F567
:1075FE00191023E87E33E518127924F5181023E8C4
:10760E007E393026027E3BE537127924F53710237A
:10761E00E3227F707E151278E7C2247E1BE51C12D2
:0A762E007924F51CD2247E21E51B0F
:10763800127924F51B1023E77E27E51A127924F521
:107648001A1023E67E2DE519127924F5191023E87E
:107658007E33E518127924F5181023E82278D7E646
:10766800C2E775F00A847866F537303B0578698596
:10767800F0371276D530262BE53775F003A40404CD
:1076880075F00584FBE51975F00AA4251875F00650
:10769800A42BFBE435F0FC125E05F537125E05F508
:1076A800188B1922E563FC339217AB625003125E04
:1076B80076305C0A7AD2125BF17840125D93AE04A0
:1076C800AF037C277D10125CFC8F1C8037E6FD33EE
:1076D80092171886041886035003125E7E7A097979
:1076E8002778C0125D908B1EADD3ACD2AB0679EA79
:1076F8007860125D8E8B1DAF06AED27C177D70123E
:107708005CFC8F1CAF05AE047C037DE8125CFC8F2B
:107718001BAF05AE047C007D64125CFC8F1AED750E
:10772800F00A84F51985F01822EC339217500312E9
:107738005E76751D30301786751D2D808178427BE9
:10774800607CEA800678407B207C4E12B4DF792783
:107758007810125D8E8B1CAF06AED280AB30262A15
:08776800E51975F00AA42518CB
:1077700075F00AA42537FBE435F0FC7A05125BE3CB
:107780008C068B077C007D03125CEF8E048F031246
:10779000769FE51E75F00AA4251D75F00AA4251C28
:1077A00075F006A4251BFBE435F0FC7A0A125BE3B6
:1077B000EB251AFBE43CFC7A0A125BF1EB2519FB82
:1077C000E43CFCE43DFD7A0A125C03EB2518FBE483
:1077D0003CFCE43DFD301703125E7EA60518A604AE
:1077E00018A60378D7E6A2E7923DC2E775F00A84AF
:1077F000FCABF0303B0EAB37EC75F00AA42BA23D8E
:1078000092E7F622AC3780F0127823305C0A7A4097
:10781000125BF178D2125D93301703125E768C639F
:107820008B62221278337A0A125BE3EB2518FBE4B1
:107830003CFC22E51C75F00AA4251B75F00AA42562
:107840001AFBE435F0FC7A0A125BE3EB2519FBE442
:107850003CFC2212788512D06FC202C223127885B6
:1078600010000810010510021B80F51031ED1030DA
:107870000D102604D22680E3D230C23180DDD23111
:04788000C23080D7BB
:10788400227F35909817126C3A90983520300F90DB
:10789400985120310990982620260390981E1F7E27
:1078A40017126C0902CFDC7F357E01909352126C63
:1078B4003C7F347E3A1279D4744E12C71F12CFDC47
:1078C40012D06FC2027F347E3AD2177511597512E5
:1078D4004E802675112E751227801E75113E751265
:1078E4002F801675112B75122D800E75114E751281
:1078F4005380067511457512571279D4E511301766
:1079040002E51212C71F12CFDC1000081001051087
:10791400020B80F5D23C1017E3D21780DF0279CF37
:107924004430F812792EE8540F22C2218002D22169
:10793400A224922292231279D4E830E709D23C742B
:1079440030302102745FF812C71F12CFDC100034EC
:1079540010010510025D80F5D23C102266102367E9
:10796400B43909745F2021DF743080DBB45F0474A0
:107974002D80D4B42D04744180CDB45A0474308065
:10798400C60480C3D23C302406102237102338B4F6
:107994004104742D80B1B42D04745F80AAB45F04D3
:1079A400743980A3B43009745A20219B74398097A8
:1079B400148094B47108D223E812C71F800DF8C252
:1079C40023800874718001E802794B9079E980037F
:1079D4009079E5C007EF2408FF12C74DD00702CF06
:0979E400DC0205F8F802050000C0
:10CF330075A70090CF6575F02D84C2D5C2D1601757
:10CF4300D2D1146007D2D514600DC2D1E5F093FCA1
:10CF5300742D95F093FB22E5F093FB742D95F093DC
:10CF6300FC220009121B242C353E474F5860687081
:10CF73007880888F969DA4ABB2B8BEC4CACFD4D9EB
:10CF8300DEE2E6EAEDF0F3F6F8FAFCFDFEFFFFFF62
:10D02100D23D8002C23DED8BF0A430E70205F0C392
:10D03100E895F020D50425F025F0FEED8CF0A43024
:10D04100E70205F0C3E995F030D10425F025F0FFA2
:10D05100203D0B2487500122EF24CC40012202D035
:01D06100E1ED
:10C99D00203A7A7E1C7F5312D0E17F5912D0E11ECE
:10C9AD007F5712D0E17F5512D0E17E2312D0E17F67
:10C9BD005712D0E11E7F5912D0E17F5312D0E11FE3
:10C9CD007E2012D0E17F5A12D0E17E1E12D0E17F7F
:10C9DD005212D0E112096EE5BD20E0143006117F30
:10C9ED00357E1C90CA5DE571700390CA6702C74D14
:10C9FD00E5716018E57012CF33781F79567D0912F5
:10CA0D00D025303A0312CA300DBD16F3227E1C7F9D
:10CA1D005390CA4612C74D200CD67E1F7F4112BDC2
:10CA2D00E580BCC0060E30D5021E1E12D0E1D00628
:10CA3D001F30D1020F0F02D0E1070700386C446C94
:10CA4D00380005052070D8702005057088A88870FD
:10CA5D00080710387CFE383838000807102844C6FF
:04CA6D00282838003D
:10BBC3009098637F717E23126C3C12096EE5BC7EF4
:10BBD3003112C6DA30121AC23C12096EE5BCFB758B
:10BBE300F00AA4F904FAC23D12B17D12BE51303DF0
:10BBF3000122DAF712BD697C00EBF4042E4019AD83
:10BC030003125CEFEFA2D1203C077E237F6502C3C2
:10BC130039AE16AF1702BD0AAD01125CEFEF12C4C5
:10BC230027203C077E237F6502C35DAE16AF170254
:10BC3300BD2E7F567E0512BD957F3D12BDA87F6F39
:10BC430012BDA87E1F7F4112BDE57E0A7F4112BE51
:10BC5300077E227F5912BE072012012212B17D8571
:10BC63007A1D855E1C857B1B855F1A7AC0C23D12D7
:10BC7300BE4D203D5212BD697C007D14125CEF74F1
:10BC8300562F20D1029F9FFF24CB40028037EF2401
:10BC93008850028030EA1475F00384FE12D0E1C3A9
:10BCA300E51B957BFEE51A955F92D55004EEF404EF
:10BCB300FEEEC313FE24E0400C741F2E30D5029E0B
:10BCC3009EFE12D0E1DAA8227F5212BCDD7F5A1207
:10BCD300BCDD75175375160080287E0012D1110E36
:10BCE300BE12F922201201227F157E2B742012C767
:03BCF3001F7F1C94
:10BCF6007E2B12D1110EBE40F975171575162DD271
:10BD06003C02BBDCC23D6002D23D92D175F0803070
:10BD16005C04F5F08001A4A2E792D5E5F075F03257
:10BD260084F8E5F075F00584C0E0E5F0A2D533C0EF
:10BD3600E0E8601E12C70CEE2406FED0E0F8D0E064
:10BD460012C70CEE2406FE742C12C71F0E0EE80254
:10BD5600C70C7420303D07742B20D102742D12C7F6
:10BD66001F80D4C3ED957AFFEC955EFE92D1500309
:10BD7600125E66227F1512BD817F327E3E12D0E1B1
:10BD8600DEFB227E0912D0E10EBE36F9227E0112BA
:10BD9600D0E10E0EBE3FF8227E3312D0E10EBE4039
:10BDA600F9227E047D1112D0E10E0E0EDDF81F1F62
:10BDB6007E3590986C305C057E31909870026C3CB4
:10BDC6007405305C097E32740112C6DA74067E365A
:10BDD60012C6DA7E3A740012C6DA7E3D02C6DA7DF3
:10BDE6000F12D0E10F0F0FDDF8227F737D03800461
:10BDF6007F727D0512D0E10FDDFA227F717D07800B
:10BE0600F37D0A12D0E10E0E0F0FDDF722203D075B
:07BE16001237907003D23DCA
:10BE1D0022056D12AF1CE4F5F7C2B2C2B2ABF7F555
:10BE2D00F7C2B2C2B2E5F7FA30E411EB251DF51DEC
:10BE3D00E4351CF51C0519EA30E3010ED2B280156C
:10BE4D00780380027801203D071237907003D23DB0
:10BE5D0022D8F3056DE56D2409F56D12AF1CE4F5DF
:10BE6D00F7C2B2C2B2ADF7F5F7C2B2C2B285F71BD7
:10BE7D00F5F7C2B2C2B2E5F7FCD2B2C220543F30E0
:10BE8D00E50244C0CC54C02323F51AE56D24F6F524
:02BE9D006D2214
:10C8C4007E017F0990C94212C74D2051097E037F22
:10C8D40000743F02C71FE4FEFFC3E54512C125FDF6
:10C8E400940AED403D9464ED4002746312C5BD7E2C
:10C8F400017F09E552240575F02D84AAF075F00531
:10C90400A4CA75F00B842A90C92D9312CF33BCB8F6
:10C91400027BB87D04EE2DF8EF2DF90D12D021DD48
:10C92400FB227E0312C70C80C6000C1622222D396E
:10C93400444F4F5A66707C7C87939EA9A9000909CD
:10C944000800410000000000888000000000410051
:10C954000800120982E5BCB4F8339004C3E0602CEB
:10C96400FA24F340277F137E0012D0E10F0F12D078
:10C97400E10E12D1111F1F12D1110EDAEC7F147EB9
:10C984000012D0E10E12D1110EBE12F5229005CC88
:09C99400E0C3941240F60480C7D0
:10C12500305D0A75F08AA42480E5F03400227F0092
:10C135002074147E110F90C1C312C74D7F0A7E0A69
:10C14500E52E540702C5D47E0BE571B4FF2DE551EC
:10C1550024025003755100E55112C12575F005A45F
:10C16500ACF0FB125BB97E0D781CE66004E612C7E5
:10C1750005EE2405FE18B818F4800612C12512C56F
:10C18500C37F0C7E11E571602F0EE57064B46028E5
:10C1950064B475F03284C0F012C705CE2405CED044
:10C1A500E075F00584C0F012C705CE2405CED0E0B9
:10C1B50023302D010402C705907D18026C09070F75
:10C1C500FFFF9EE7AD6B9C6BAD6B9D67FFFF7554E5
:10C1D5008030745F78BD79BBE6FC27FB1819E6FD56
:10C1E50037F9EBF87B00125D958B547F087E11A81B
:10C1F5000690C23912C74D30101120730E7F0A7E8A
:10C205001712D1110E0E12D1117F08E5542483E5C2
:10C2150054500224FA75F01984FB90C2419328FE0C
:10C22500EB90C24B93FD12D0E10F0F12D0E11F1F0F
:10C235000EDDF322030F0100FFFE03800000000066
:10C2450007070D0C0B0A050403020101020304058F
:10C25500306701227F357E00746F12C71FE57E604F
:0DC26500F212C12575F06484F87E06E5F044
:10C2720012C622E860E07E0002C70C202C01229048
:10C28200C28702C74D050EFFF0E01CF004F81CFF48
:10C29200F0301201227F6E7E0090911712C74D7FFF
:10C2A2001512BD817F1F12BD817F2912BD817F17AB
:10C2B2007E06E53F30E00B909880305C03909894C6
:10C2C20080132074077E0190913780099098753011
:10C2D2005D0390988A126C09307306E54E60021570
:10C2E2004E205718E54EB40113120991C3E55C952F
:10C2F20060F5BCE55D9561F5BD1248EB7F217E01DD
:10C30200E53F30E02130570590920C8016E54E70E3
:10C3120005909218800D909143126C097E30E54E83
:07C3220002C628126C09227B
:10C48F00125B8B7F207E05751900781DC2D5E630B3
:10C49F00D51712C705EE2405FE18B818F17E1F74C4
:10C4AF0063305C02746502C71F7005B8191880E20B
:10C4BF00D2D5CE24FACE746B301702742D12C71F4B
:10C4CF00EE2406FE80C8742012C71B80C8781C801B
:10C4DF000D7F007E23AC5EAB7A125B8B781DC2D5CD
:10C4EF00E630D50C12C70CEE2406FE18B818F12250
:10C4FF007005B8191680EDD2D53017E4CE24FACED8
:10C50F00742D12C71FEE2406FE80D5742012C71F8C
:10C51F0080D5125B8B781DC2D5E630D51612C6DAE0
:10C52F00EE2404FE18B818F10E745E305C02742706
:10C53F0002C6E97005B8191680E3D2D53017DACEE6
:10C54F0024FCCE742D12C6EDEE2404FE80CB742095
:10C55F0012C6ED80CBC23D12C5770F0F0E0E74635E
:10C56F00305C02746502C71F125B8B781DC2D5E663
:10C57F0030D50C12C73CEE2408FE18B818F1227003
:10C58F0005B8191680EDD2D5301716740BCE24F8D6
:10C59F00CE12C73CEE2408FE80D5740C12C73C8027
:08C5AF00D5303DCB740A80E594
:10CA71007F797E24E55F30E70122AC5F1CAB7B123E
:10CA81005BB9E51B700E742012C71FEE2405FE1260
:10CA9100CABF800C12CABFE51B12C705EE2405FEF2
:10CAA100E51A12C705EE2405FE742C12C71F0E0EDF
:10CAB100E51912C705EE2405FE745E02C71F742D29
:10CAC100201702742B12C71FEE2406FE22E55F30E9
:10CAD100E70122AC5F1CAB7B125BB9E51B700E74E6
:10CAE1002012C6EDEE2404FE12CB18800C12CB18D6
:10CAF100E51B12C6DAEE2404FEE51A12C6DAEE24AC
:10CB010004FE742C12C6ED0E0EE51912C6DAEE24DF
:10CB110004FE742A02C6ED742D201702742B12C66E
:06CB2100EDEE2404FE22EB
:10C329007F097E2530040512C4238028A275E5798A
:10C33900C23D6002D23D92D175F080305C04F5F0C7
:10C349008001A4A2E792D5E5F075F03284F8E5F012
:10C3590075F00584C0E0E5F0A2D533C0E0E8602AB5
:10C3690012C73CEE2408FED0E0F8D0E012C73CEE3C
:10C379002408FE0F0FE52B5403701F746012C71FAA
:10C389001F1FEE2404FEE802C73C740C303D0674FE
:10C399000A20D1010412C73C80C9205904742E8097
:10C3A900DC205804746180D5746280D13004051290
:10C3B900C4238028A275E579C23D6002D23D92D19D
:10C3C90075F080305C04F5F08001A4A2E792D5E510
:10C3D900F075F03284F8E5F075F00584C0E0E5F019
:10C3E900A2D533C0E07F3E7E1CE8602012C79DD0F5
:10C3F900E0F8D0E07F3E7E2812C79D7F447E3274EC
:10C409002E12C71F7F3E7E37E802C79D303DE0747C
:10C419000A20D1010412C79D80D59005CAE075F0A4
:10C429000A84F8E4C5F0C2D522301105E54AB40200
:10C4390050C39006E9E0957AFB9006E8E0955EFC2A
:06C449005003125E76ECC8
:10C44F00C31360047B63800FEB13FB249C40F52424
:10C45F004F4004C20480079005CAEBF0D204900647
:10C46F00E6E09006E8F09006E7E09006E9F0E55E7A
:10C47F009006E6F0E57A9006E7F02212C46D80DEB2
:10BE9F00E54424F64001227800E552206607C39559
:10BEAF0070500224B40475F00384F9E928FE24C409
:10BEBF005001FE12BEE112BEED1E12D0E1C3E99891
:10BECF00FE5003243CFE12BEE11E12D0E108B81F43
:10BEDF00DA22EE2420FE24C250032402FE22E8249C
:10BEEF00F1E8C2D55006D2D5E8F4241F23FF90BF46
:10BEFF006F93CF0493FAE545F5F0A4ACF0FB125C19
:10BF0F001AE544F5F0A49BFBE5F09CFCEB2420FB29
:10BF1F00EC3400FC12BF50FAE5458FF0A430E70275
:10BF2F0005F0E5F020D502F4042A75F00520190379
:10BF3F0075F00384FF24DF50027F20C374329FFF0C
:10BF4F0022EC24F0500BEB2460EC340090BFBF9335
:10BF5F0022EB33FBEC33FCEB33EC3390BF8F9322AC
:10BF6F00FF00FF03FA0BF318EA2ADE40CF58BE7327
:10BF7F00AB8D96A880C068D64FE835F51BFD00FF46
:10BF8F0000080B0E101214151718191B1C1D1E1F5D
:10BF9F0020212223242526262728292A2A2B2C2D27
:10BFAF002D2E2F2F3031313233333434353636375F
:10BFBF00373839393A3A3B3B3C3C3D3D3E3E3F3FBB
:10BFCF004042444648494B4D4E505253555658598E
:10BFDF005B5C5D5F60616364656668696A6B6D6E0B
:10BFEF006F7071727374767778797A7B7C7D7E7FD0
:10BFFF00808182838485868788898A8B8B8C8D8EBE
:10C00F008F9091929394949596979899999A9B9CC7
:10C01F009D9E9E9FA0A1A2A2A3A4A5A6A6A7A8A9E4
:10C02F00A9AAABACACADAEAFAFB0B1B1B2B3B4B413
:10C03F00B5B6B6B7B8B9B9BABBBBBCBDBDBEBFBF4D
:10C04F00C0C1C1C2C3C3C4C5C5C6C7C7C8C8C9CA92
:10C05F00CACBCCCCCDCECECFCFD0D1D1D2D2D3D4E0
:10C06F00D4D5D5D6D7D7D8D8D9DADADBDBDCDDDD36
:10C07F00DEDEDFDFE0E1E1E2E2E3E3E4E5E5E6E691
:10C08F00E7E7E8E8E9EAEAEBEBECECEDEDEEEEEFF3
:10C09F00EFF0F1F1F2F2F3F3F4F4F5F5F6F6F7F75A
:10C0AF00F8F8F9F9FAFAFBFBFCFCFDFDFEFEFFFFC9
:10C0BF00E54524FD400122E552206607C3957050E7
:10C0CF000224B40475F00384241FFE24C2500324F9
:01C0DF00025E
:10C0E000FE12C11AEEFD241EFE24C250032402FEDD
:10C0F00012C11AE544240275F00520190375F003F6
:10C1000084F4042432FF24EE500F12C10FAE051E3A
:10C110001E7C0512D0E10EDCFA227F1512D0E10F51
:05C120000FBF2DF82205
:10C7DC007E00206615E5700475F0B484E5F075F004
:10C7EC000384FE6004C3743C9EFE745312C8077429
:10C7FC005712C807744E12C80774457F2F12C6ED26
:10C80C00BE00077E3C12C6ED7E00EE240875F03C9F
:10C81C0084AEF00F0F0F12D0E10E12D0E10F12D038
:10C82C00E11E12D0E1EE240775F03C84AEF022300C
:10C83C00745C301259E54AB4040122B4060122E5B5
:10C84C007112BF398F057C037E1E30662AE5700499
:10C85C0075F00384241EFE24C6501C24FB500424B3
:10C86C00038013C00612C883D0E024C67C01600686
:10C87C000C1460020C14FE12C88F0EEE24C1400280
:10C88C00DCF5228D0712D0E10FEF24CE50F722E514
:10C89C0053206607C39570500224B40475F00384CA
:10C8AC00241FFE24C250032402FE12C8BA0E7F239A
:08C8BC0012D0E10FBF2DF9229B
:10CF9300AF177E00E53C12C5B77E0C742E12C71F77
:10CFA3007E12E53B12C5B77E1E742E12C71F7E2468
:10CFB300E53A02C5B77E0E78ADE612C6227E187436
:10CFC3002C12C71F7E1B18E612C6227E25742C1254
:09CFD300C71F7E2818E602C622E1
:10D0A2007F797E16743B12C71B7E18E53F12C6229B
:10D0B2007F797E0078AEE612C6227E0A743B12C7E2
:10D0C2001B7E0CE53E02C6227F797E00E54012C639
:0FD0D200227E0A743B12C71B7E0CE54102C62268
:10CC8400787512CCD47453201702744E207406E5C0
:10CC94002E54074430AF1712CCFE7E3BE57DC454BE
:10CCA4000F12C70C2074077E07742012C71F7878F0
:10CCB40012CCD4E5172409FF7457201702744520B9
:10CCC4007402742012CCFE7E3BE57D540F02C70C27
:10CCD400E6FD339217188604188603301703125E94
:10CCE4007E79177870125D8E8B13AF06AED27C00FE
:10CCF4007D64125CFC8F148D15227E0012C71F7E8A
:10CD040007E51312C5D47E19746412C71F7E20E58B
:10CD14001412C5B77E2B742E2073030E742C12C705
:08CD24001F7E2FE51502C5B7C3
:10CE4500E54A602E7A2420E00E7A26141460087ACA
:10CE550028141460027A297F717E00EA12C71F2008
:10CE65005505205406800B745B8002745C7E0012AD
:10CE7500C71F20110778A9B60007802F30262CC2BE
:10CE8500269099BC7F68126BF77F66A85AE54AB46D
:10CE9500060108E875F06484740AC5F084C0F012D0
:10CEA500C73CEE2409FED0E012C73C20080FE53749
:0ECEB500640260097F367E2E744112C6ED22A3
:10CB270020144F740512D188EF33EE33F9EF030366
:10CB3700541FF5F090CB7AE993A4C5F013C5F01311
:10CB4700C5F013C5F013C5F0135403FCE5F013FB50
:10CB5700E9242093C9244093C39BC4540FFBE99C49
:10CB6700C4FC540FF9EC54F02B2446F57BE934F65A
:10CB7700F55F22FFFFFFFFFFE6C5AD9C8F857D7741
:10CB8700726E6C6A696A6A6C6F747A828D9DB4D9A9
:10CB9700FFFFFFFAE9DCD3CEC9C6C3C0BEBBB9B736
:10CBA700B5B4B2B0AFADABAAA8A6A4A2A09E9C99FB
:10CBB70096918C00381CE735D137246F00C5B3C177
:10CBC700E61F66B60E68C21867AADBF4EDB94675AC
:03CBD70010A200A9
:10D16800D2A27408D2A1D2A300C2A3C2A1D2A300A2
:10D17800C2A3D5E0EF7405D2A300C2A3D5E0F8227C
:10D14100C2A3D2A2D2A1D2A300C2A375F008339286
:10D15100A1D2A300C2A3D5F0F5C2A175F003D2A359
:07D1610000C2A3D5F0F82283
:10B7E80012D141D2A300C2A3C2A175F008E4D2A32A
:10B7F80000C2A3A2A233D5F0F5FE75F008E4D2A3E7
:10B8080000C2A3A2A233D5F0F5FFD2A300C2A3229F
:10B81800E478806608B88BFB70012274D512B7E80B
:10B828007881C3EE13FEEF13F692D118EE2460F67A
:10B8380074D612B7E87888EF33CE33CE33CE33CE12
:10B8480033A2D192E25407FCEEFB7A08125BE3ECD8
:10B85800244FF608EBF674D912B7E8EF543F788214
:10B86800F67886EF33CE33CE33CE33CE335403F669
:10B8780008EEF618161608E6C4FF54F0F618E6C4E3
:10B88800CF540F2FF674DA12B7E8EF232354FC785D
:10B8980083F67884EEF608EF54C0F67880E46608FC
:10B8A800B88AFBF62212B7F07889C3EF96FF18EE34
:08B8B80096FEA2E79216501063
:10B8C000125E66740FF8F9125C30EF2CFFEE3DFE4D
:10B8D000788BEEF608EFF622E6182016072CF7E62E
:10B8E0003D19F722C39CF7E69D80F66A405E8056BC
:10B8F000E050F04B0044803DC0384031D02BA025B3
:10B90000601F2018D014000F000AA0014401580144
:10B91000680178018801A001B401D001EC02100295
:10B9200038026802A002DA030C034D78BE8020853D
:10B930008E8A9D8F4D95BA9A97A0BEA631AC53B210
:10B940002AB801BD6AC1EDC4D1C78812B7F0788D9D
:10B95000EEF608EFF67887798C125C307883799070
:10B9600012B8D87885798C125C307881799212B8C7
:10B97000D8788DE624E4FE08E63392D13392D5548C
:10B98000FCFFEEA2D133A2D533FE780F7992125C80
:10B990003078947990C3EC97F61819ED97F679946E
:10B9A00090B8EB7F1F7D11EF93C3971F19EF93970B
:10B9B0001F091DED600240EF0F90B90B798DEF93D9
:10B9C000F7090FEF93F7788E7994125C3090B92BCA
:10B9D000EF93C39BFB1FEF939C2420FC7897E62BEF
:10B9E000F618E63CF618E436F6740612D188D2371B
:09B9F000EE24F740062402500287
:10B9F900C237EEFCEFFD740712D188C3ED9FFFEC4F
:10BA09009EFE78B7E6FD337C0050011CEF2DFFEE5A
:10BA19003CFE78D8E6C4540F2FFFE43EFE789CEF35
:10BA290026F618EE36F62220141220370F789DE6F6
:10BA3900B4050912BAE812BB1D12BB662220145EB6
:10BA49007897799A12BB81125DEEC3EE9420FE922B
:10BA5900455003125E667C007D05125CFC3045038F
:10BA6900125E66E531B40C3612CC6A120987E5BC60
:10BA79002FF560E5BD3EF56120E71124F8500DFA78
:10BA8900C3E5609AF560E5619400F561120991E5F5
:10BA9900BC2560F57AE5BD3561F55E12CC777897FE
:10BAA900799AC3E697FB1819E697FC7A02125BE3C9
:10BAB90030370B7A02125BE3ECFEEBFF800312BA1C
:10BAC900E812BB1D20140312BB6678957998E6F736
:10BAD90076000809E6F776000809E6F77600227984
:0CBAE9009CE77700FB19E77700FC789DD4
:10BAF500E6B40506EB33FBEC33FCECA2E792D5503C
:10BB050003125E767A32125BF1ECFBEDFC30D50365
:10BB1500125E76ECFEEBFF22EE2408FE740420375D
:10BB2500167406307511789DE6B40504740C80070B
:10BB3500F42406C323540FFD7C00125BCF789FE6E7
:10BB4500FC08E6FBC374109DFA125BF1EFF8EEF901
:10BB5500125DEEE878A02FF6FF18EE39F62480FE88
:10BB65002292754003125E66EF33EE33F579C276A5
:10BB7500307508E57924F15002D27622E627FB18C4
:10BB850019E637FC1819E637FD2212B1247F08782B
:10BB950071793A12BBAA0245AD855E63857A6278F2
:10BBA5007379647F06E6F70809DFFA22786479730A
:0EBBB50080F1787379AF80EB78AF797380E51B
:105B6900E4FEFFFC7D0A791DE7540F2FFFE43EFE9A
:105B7900B91902800619125BCF80ED301703125E46
:105B89006622305C2BEC3392175003125E76EC24BC
:105B9900D950047C277B007AD2125BF1EB33CC33EA
:105BA900CD33CC33ED33FBEC33FC301703125E7687
:105BB900EC3392175003125E767919125E05F709D4
:105BC900B91DF8A70322EFF88DF0A4FFEDC5F0CEBB
:105BD900A42EFEEC88F0A42EFE22EB8AF0A4FBE5AD
:105BE900F0CC8AF0A42CFC22EB8AF0A4FBE5F0CCE3
:105BF9008AF0A42CFCE435F0FD22EB8AF0A4FBE545
:105C0900F0CC8AF0A42CFCE435F0CD8AF0A42DFD6B
:105C190022EB8AF0A430E70205F0E5F0CC8AF0A483
:105C29002CFBE435F0FC2286F0E7FDA4FAABF01971
:065C3900E786F0A42BFB3E
:105C3F00E435F0FC18E68DF0A42BFBEC35F0FCE41A
:105C4F0033FDE687F0A42CFCED35F0FD22EB89F057
:105C5F00A4CBAEF08AF0A42EFEE5F03400FDEC8963
:105C6F00F0A42EFEE5F03DFDE433CC8AF0A42DFD2B
:105C7F00E5F03CCEFC22EB89F0A4CBAFF08AF0A488
:105C8F002FFFE5F03400FEEC89F0A42FFFE5F03E86
:105C9F00FEE433CC8AF0A42EFEE5F03CFCED89F057
:105CAF00A42EFEE5F03CFCE433CD8AF0A42CFCE5F9
:105CBF00F03D8E058C068F04FF22C2D5EC30E70530
:105CCF00B2D5125E6EEE30E70DB2D5125E66125C83
:105CDF00FC125E6E8003125CFC30D503125E6622EE
:105CEF00C3EC13C0E0ED132FFFD0E03EFEBC000B62
:105CFF00BE0029EF8DF084FFADF022E4CCF975F0F2
:045D0F0008EF2FFF6B
:105D1300EE33FEEC33FCEE9DEC994005FCEE9DFE6C
:105D23000FD5F0E9E4CEFD22EDF9F5F0EE8420D2B3
:105D33001CFEADF075F008EF2FFFED33FD40079922
:105D43005006D5F0F222C399FD0FD5F0EA22EC33C9
:105D5300EE3400FEEF3400FF7D007A00790078090D
:105D6300C3ED9AFDEE9BFEEF9CFFB392D54009ED88
:105D73002AFDEE3BFEEF3CFFA2D5E933F9ED33FDFF
:105D8300EE33FEEF33FFD8D92279007A00C38015B2
:105D930079007A00C3EA13FFE913FEE8132BFBEE45
:105DA3003CFCEF3DFDE4F5D2F5D333FE7F19C3EEA2
:105DB30098FEE5D299F5D2E5D39AF5D3B392D540BF
:105DC3000DEE28FEE5D239F5D2E5D33AF5D3A2D5C7
:025DD300EB33B0
:105DD500FBEC33FCED33FDDF0122EE33FEE5D23380
:105DE500F5D2E5D333F5D380C3EDC454F0FEECC44E
:105DF500FF540F2EFEEF54F0FFEBC4540F2FFF227C
:105E0500EC75F00A84FCEB54F025F0C475F00A84B7
:105E1500C4CBC454F025F0C475F00A842BFBE5F01F
:105E250022AC10AB11125E05A904AD03FA7C197BF7
:105E350099125BE3AE04AF03EA75F006A4F8AC1261
:105E4500AB13125E052875F00A8485F014F8EF2B64
:105E5500FFEE3CFEEF28FFE43EFEE43DFDE439FCA9
:105E650022C3E49FFFE49EFE22E4C39DFDE49CFC67
:105E750022C3E49BFBE49CFC22C3E49BFBE49CFC67
:105E8500E49DFD2275D4107B807A0079807800EA44
:0A5E9500F5F0A4FCADF0EBF5F0A46D
:105E9F00FEAFF0EB8AF0A4C333C5F033C5F092D553
:105EAF002DFDC5F03EFEE430D501043FFFB5150DC5
:105EBF00EEB51409EDB51305ECB51201224006EA53
:105ECF0098FAEB99FBD5D40ABB0001220ABA00015C
:105EDF000B22C3E913F9E813F8EA28FAEB39FB8030
:105EEF00A478087B807D807C00EDF5F0A4FAE5F0C6
:105EFF008EF0B5F007EA8FF0B5F001224003ED9B6D
:105F0F00FDD827BDFF0122EDF5F0A4F9A8F0ED04AF
:105F1F00F5F0A4C399FAE5F09813CA1329F9E83AF2
:105F2F00F8C3E99FE89E50010D22C3EB13FBED2B45
:105F3F00FD80B67473F8F9E627FB0809E637FC080D
:105F4F0009E637FD30E703125E7EEB33FBEC33FCE3
:0B5F5F00ED3323FD242083F8ED241C0B
:105F6A0083FFED241883FAED241483F9EF99F9E8F5
:105F7A009AFA125C5CEF9DFFE89EFE22FFFFFFB6D5
:105F8A00FED7FD63FB5DF8C4F59BF1E3ED9EE8CF18
:105F9A00E379DD9ED743D06BC919C153B91CB079D7
:105FAA00A7709E06943F8A237FB674FF6A045ECB6D
:105FBA00535B47BB3BF1300423FB17DE0BB2C21D18
:105FCA00C232532CF8C3E5679576FBE5689577FCF2
:105FDA00E5699578FD30E705D261125E7E24F050BE
:105FEA000312609CAA06A907125C85EC2480E43D92
:105FFA00FBF9F51AE43EFCFAF519E43F6002D232E5
:10600A00125C5C8B128C138D148E15C3E564957328
:10601A00FBE5659574FCE5669575FD30E705D2628A
:10602A00125E7EEBF9F51FECFAF51DED6002D23235
:10603A0030320122125C5CEB2512F512EC3513F5B5
:10604A0013ED3514F514EE3515F51540E1025E89A8
:10605A00125FC820323BEB242E40D3EA2401CB3412
:10606A0000FC7A07793D125C5CC010C0118E108D5D
:10607A00118C128B13E4FCFD7E077FD012A8E685F3
:10608A001203851302D011D010BB0005BA0002D248
:10609A001D22B261C374809BFB74F59CFC74209D25
:0160AA00FDF8
:1060AB0022204D7D20487A303F777F747E0112BDD0
:1060BB00957E1F12BE0175A7009004EDE0A2E7923A
:1060CB00171392E7FC1582E013FB301703125E7671
:1060DB00BC004EEB604B20E74820E64510E5132053
:1060EB001707C3741F9BFE80027E1F12BDF60EDBCB
:1060FB00FA22FB2017097E00C374209BFB8008EB60
:10610B00241FFE74209BFB12BDF00EDBFA2275A739
:10611B0000758307E559C4440FF582E0A2E792525C
:10612B00222212BBB7126119C2E775F00A84FEAFC7
:10613B00F075A7045382F1786412619AAE07786701
:10614B0012619A75A700E57DC4540FFEE57D540FCF
:10615B00FF787312618EAE07787612618E74AF1270
:10616B005F4412605A120982E5BD75F00AA4F9EA80
:10617B00999004ECF0A3EB95F0F0A2E7923DD23F9F
:10618B0002BBBD860308860408860518188006E046
:10619B00FBE0FCE0FD7A0A125C0320E70CEB2EF629
:0E61AB0008E43CF608E43DF622C3EB9EF6083D
:1061B900EC9400F608ED9400F622C2338006204DD7
:1061C900F92048F6C23F302A0F78A87600223038E5
:1061D900FCC23878C5864622E54824F640EFE558E2
:1061E9000460EA75A700758307E559C42408F58298
:1061F900E070DB0582E0FFE54A64046015E54A6466
:1062090006600F801DEF24BE5029C23878C5864626
:10621900802175390AEF20E70975390520E60375EC
:1062290039022038E0EF24C34009D23878C5A646A0
:10623900754600120982E5BD240DC39F40251261F0
:106249002D303D1F753901204006D24078A87623AC
:1062590020522CE55965586026204D23204820D22C
:1062690033801C303319204D1220480F1285BE058A
:1062790059C3E55895595003855859C233C240222C
:10628900E558B4FF012285581175A704758307E500
:106299004824F65002805C201259202905202A0240
:1062A900805112BBB7E4F516F51775100012631586
:1062B900E510700312BBB112632E302910E51B25BE
:1062C90017F517F51BE51C3516F516F51C12633B7A
:1062D90012BBB10510C3E511951050D175A7000285
:1062E900BBBDE55AF51124F6500375110A75A704CB
:0362F900758306A4
:1062FC0075100012631512632E12633B0510C3E573
:10630C0011951050EE75A70022E510C4F582E0E05F
:10631C00F564E0F565E0F566E0F567E0F568E0F555
:10632C00692275A7011266891239F775A70422E94B
:10633C00F0E51CF0E51BF022E510C454F0F582E00A
:10634C00F512E5822406F582E0F511E0F51CE0F586
:10635C001B22202845E558B4FF012275A70475833C
:10636C0007E559F5103033066558600205101263C5
:10637C0044E0F513E07F797E3D12C6EDE5137E39DE
:10638C0012C6EDE5127E3512C6ED30480B7F7F7ECE
:10639C003512D0E10EBE40F9802C2012012275A7D7
:1063AC0004758306855B10126344E512700B7E3A0C
:1063BC007F79745D12C71F800D75F06484E5F07EE3
:1063CC00397F7A12C66FE537B402051284428045D4
:1063DC00B403028040E51C7006E51B24FB5036E537
:1063EC0011F964B4602F20062CE537600D200C0ADF
:1063FC00C3E99570F9500324B4F9E912CF33781D31
:10640C0079547D1D90CA4FE53F20E00390CA561287
:10641C00D02512C74D75177975161912646D75A7AD
:06642C00009006E3E511FB
:10643200F0A3120982E5BC75F01970040475F0141A
:10644200A4951BFBE5F0951CFC92245003125E768A
:10645200ECF0A3EBF0C24FC263EC700EEB24E6400B
:1064620002D24FEB24C84002D26322E51C24ED4045
:106472002BAE1CAF1B1266537C007D32125CFCC03B
:1064820005EFAF17AE1612C628CE2405CE742C1215
:10649200C71F0E0ED0E02312C622801B12664A12BC
:1064A20064C7CE2405CE742C12C71FCE2402CEE8B8
:1064B20075F0058412C705CE2404CE7422305D0225
:1064C200746602C71FEE243D50047EC37F4B7C01DD
:1064D2007DF4125CFCC004C005EF6007AF17AE1676
:1064E20012C628D007D0067C007D32125CFCA805BB
:1064F200EFAF17AE16CE240ACE02C70512664AEED9
:106502002450305D03EE24A150047EC37F4B7C01F6
:106512007DF4125CFCC004C005EF6007AF177E2F4C
:1065220012C675D007D0067C007D32125CFCC00515
:10653200EFAF177E3712C6DA7E3B742C12C6ED7EA1
:106542003DD0E075F0058402C6DA304803207401BC
:0265520022E441
:10655400FCF5A79006E3E0F9A3E0FE24FE40EFA3D8
:10656400E0FF7D78E537600B304FE3200C2F126697
:1065740040802A12096EE5BD20E00F204F07E54652
:1065840070083063C9D206126640204F107D3CE586
:1065940046600A7D141460057D0A1470B1891112D5
:1065A4005BCF7D6F125CEFBE00A4EF24E2409FAD91
:1065B40007E51112CF33202404B2D5B2D1781F7964
:1065C4005612D025A806A907E511242D75F0B48428
:1065D400E5F012CF337407304F02740EFDFA12D077
:1065E40025B2D5B2D112D025B2D5B2D1DDF0AD02EB
:1065F40012D025850616850717B2D5B2D112D0253B
:1066040085061E85071F7A03304F027A06E511249A
:106614001675F0B484E5F012CF33A816A917AD02AD
:1066240012D025DDFBE51124EA400224B412CF3355
:10663400A81EA91FAD0212D025DDFB22C3E9957067
:10664400500224B4F922E51B2402FFE4351CFE3079
:106654005D1ABEC305BF4D028012AC06AB077A1BA0
:10666400125BF17832125D93AE04AF032278737932
:1066740064125F4612605A751CC3751B4B203204AA
:0E6684008B1C8A1B2212667130320122AC1967
:10669200AE1AA91DAF1FB90005BC00028010C3E9E4
:1066A20013F9EF13FFC3EC13FCEE13FE80E8BF29CE
:1066B200005006BE2900500122C3EF13FFC3EE13A0
:1066C200FE80EB3E7FE3E3E3E3E3E3E3E3E3E37F45
:1066D2003E0C1C3C7C7C1C1C1C1C1C1C1C7F7F3E1E
:1066E2007FE3E3E3070E1C3870E0E3FFFF3E7FE346
:1066F200E3030F0E0F03E3E3E37F3E070F1F3F7732
:10670200E7E7FFFF0707070707FFFFE0E0E0FEFFFD
:10671200030303E3E37F3E1E3F73E0E0E0FEFFE39B
:10672200E3E3E37F3EFFFFE3E30303070E1C383896
:106732003838383E7FE3E3E37F3E7FE3E3E3E37F02
:106742003E3E7FE3E3E3E37F3F030303E77E3C0058
:106752000000181818FFFF181818000000000000A9
:10676200000000FFFF0000000000003FF0000038C2
:106772001C38F00180C1F020F0FC0038F03FE0004E
:106782000000007CC6C6C6C6C6C6C6C67C18387817
:106792001818181818187E7CC6C60C183060C0C6A7
:1067A200FE7CC6C6061C0606C6C67C0C1C3C6CCC0F
:1067B200FE0C0C0C0CFEC0C0C0FC0606C6C67C3C1F
:1067C20066C0C0C0FCC6C6C67CFEC6C6060C183073
:1067D2003030307CC6C6C67CC6C6C6C67C7CC6C641
:1067E200C67E060606CC78000018187E7E181800B1
:1067F20000000000007E7E0000000000000000009B
:106802000000000000000000000000000000008006
:1068120080A0C0A000304020C08080C0A0A00000A6
:1068220060A0600000A040A05098D090882050A89E
:1068320050888850A8502060806000000040E040EE
:106842000000000000800000E000000000000040A6
:10685200002040800040A0A0A04040C04040E0C0D6
:106862002020C0E0E0204020E02060A0E020E0C046
:106872002020C06080E0A0E0E020404040E0A0E0B6
:10688200A0E0E0A0E020C0004000400000800080C6
:10689200002060E0602000E000E00080C0E0C080F6
:1068A200E0E0E0E0E0000000000040A0E0A0A0C0C6
:1068B200A0C0A0C040A080A040C0A0A0A0C0E08016
:1068C200C080E0E080C080806080A0A060A0A0E0E6
:1068D200A0A0E0404040E0202020A040A0A0C0A016
:1068E200A080808080E0A0E0A0A0A0A0E0E0E0A0E6
:1068F20040A0A0A040C0A0C0808040A0A0C060C0B6
:10690200A0C0A0A060804020C0E040404040A0A0C5
:10691200A0A060A0A0A0A040A0A0A0E0A0A0A04035
:10692200A0A0A0A0404040E0204080E02020A8702D
:10693200202070A8202008F030D0100000F0A8A875
:10694200000000E000000090204870889898400005
:10695200E0E0E000A0E0E0E0406030103060404065
:10696200E040406090909090906020602020202035
:1069720070609010204080F06090102010906010A5
:10698200305090F01010F080E01010906060908015
:10699200E0909060F0102020404040609090609025
:1069A200906060909070109060C0E0F0F8F0E0C0ED
:1069B2000000000000000000000000000000506025
:1069C2005000707050000078807008F000F88888DD
:1069D20088F800C0C8102040981800C0B098B0C015
:1069E20000602040000000000090D8FCD890000019
:1069F200246CFC6C24000020A870A8200000202039
:0D6A0200F8202000000000000000800000CF
:106A0F0000F000000000000000006060000810208F
:106A1F00408000708888888888702060202020201F
:106A2F0070708808102040F8F81020100888701037
:106A3F00305090F81010F880F008088870304080BF
:106A4F00F0888870F808102040404070888870885F
:106A5F00887070888878081060006060006060003F
:106A6F0000008000008000002040F840200000005F
:106A7F00F800F80000002010F810200070880810AF
:106A8F002000200000000000000070888888F8882F
:106A9F0088F08888F08888F070888080808870E01F
:106AAF009088888890E0F88080F08080F8F8808067
:106ABF00F0808080708880B8888878888888F88887
:106ACF0088887020202020207038101010109060BF
:106ADF008890A0C0A09088808080808080F888D81F
:106AEF00A8A88888888888C8A8988888708888887F
:106AFF00888870F08888F080808070888888A89057
:106B0F0068F08888F0A0908870888070088870F886
:106B1F00202020202020888888888888708888886E
:106B2F0088885020888888A8A8A850888850205026
:106B3F00888888888850202020F80810204080F806
:106B4F0000CCAC9CACCC0000CCD4E4D4CC0004780A
:106B5F001828C800FC40A040182020180000000092
:106B6F000000F800000000A040A0000000600060DE
:106B7F0060006000600060600000F0A8A8A8A82076
:106B8F005020000000005090B890D0908860505076
:106B9F0000707050805048FC485080304C5C6060F2
:106BAF00603C00E0F0080808F88044485C484480E6
:106BBF00008820208870000080C0A090F800304826
:106BCF00B4B44830003048B4B44830FC0098D020FA
:106BDF0058C8008080F088888888F8E8D880D8E87E
:086BEF00F8404050F85040400E
:0300000002005E9D
:03000B0002A976D1
:0C000E00206E06859950D26E32D26F32FF
:0E00230010990AC298206DE385994FD26D3274
:10003800E4F537F534F52F12D098C229C22AC268E0
:09004800C227C214C2150227B838
:03005B00022588F3
:10A969008530F0C5F065308530F060F722C0D0C081
:10A97900E0C0F0C0A775A700C083C08275D0087574
:10A989008A00300503758A7A758CEA0532E53270DA
:10A999000215320530E530640A6026201520E531BC
:10A9A900B40C0BE530B4010612AD7712CB27E531B3
:10A9B900B4180BE530B4060612AD7712CB2702ABFB
:10A9C90081C2AFD2C075C07AD2AFF5300531E53159
:10A9D90064197047F53120152AC22C7D0A740412B6
:10A9E900D188EF33EE339005CCF0EE24F5401424F2
:10A9F90002400E24014008202005DDE1022588D20D
:10AA090025D22CE5A6600215A678B5E66001167870
:10AA1900B6E660011678D8E6600116302E09E536EB
:10AA29007005C22E12ACF9E5367004C24B800215CE
:10AA39003678A9E660011678A8E66001160535E5BD
:10AA49003570021535E590307B0B30E008D278C2BD
:10AA59007BC200801A307C0B30E108D279C27CC2FB
:10AA690001800C307D0930E206D27AC27DC202E54E
:10AA79009044F8F47003753500E533600515330229
:10AA8900AB26E590F45407700302AB26A2E09200CE
:0BAA9900A2E19201A2E2920230100341
:10AAA40020144275330820001B20100C201109804B
:10AAB40013E59030E10E8006E53724FC40F3E543CE
:10AAC400541FF53320100375A6FF78A8E6705320B1
:10AAD4002E50301004E536704920100C201109E581
:10AAE4003524F55003753304D21BD2A5D2A612AC7B
:10AAF400F975B44075B24005342027262068232018
:10AB04002920202A1DA21072115017E52054076035
:10AB140011E5342438400B200026200119D27D751C
:10AB240034C8201558E531702412D16874E812D164
:10AB340041802A02AC40E53724FC40E6D27C80DF29
:10AB44003011DFE53724FC40D9D27B80D275F00385
:10AB540084E5F070DE12B8AD74E812D141E531B489
:10AB6400060512BA308016B40C0512BA46800EB42B
:10AB7400120512BA308006B4180312BA46E59030B2
:10AB8400E10530E202800620100D20110A78A8E6C3
:10AB9400705120103C80612027F32068F02029EDBB
:10ABA400202AEAE534243040E4240750E0600B20F6
:10ABB4005E088590F020F202740190ABCE93D2A58A
:10ABC400201002C2A512ACE48053C8A08269554685
:10ABD40046E536602324AA500AE53675F01984E563
:10ABE400F06027D2A6201002C2A6D2A57418304B5A
:10ABF40002746412ACE48025E52B5403600C20102D
:0AAC04000E301106E54A64026005F7
:10AC0E0012ACFF800312AC58101B08A25892A5A2DA
:10AC1E005992A675A700D082D083D0A7D0F0D0E0ED
:10AC2E00D0D020200C201009C5A67003022588C59F
:10AC3E00A632C218B40202D21812B94B30180874D8
:10AC4E00E412D14102AB6102AB5C78A7E5B46009B6
:10AC5E0024E04005760002ACFFE534702920412245
:10AC6E0020751F300D1CE57924CE40167AFFE5B114
:10AC7E0010E7010A2325B3F5B3EA35B4F5B4C313CF
:10AC8E00F5B2E660021622C241307575E57960595B
:10AC9E00206502C21CD265FF24B050027F4F75C7DB
:10ACAE000375C6FC75B901E5BFC39FF5F0A4ACF002
:10ACBE00AAF0FBF9125C5CED33CE33CE33CE33CE3D
:10ACCE0033CE33F624FA40027605301C24E5BEC39B
:10ACDE009FF5F0A4C5F0C21C79AA770375B300F5F1
:10ACEE00B4C31375B100F5B222C26578A77680D2CF
:10ACFE004179AA7703D21CE4F5B3F5B4F5B1F5B2F8
:10AD0E0022C265E57924CE50097628301CE37446BC
:10AD1E0080C4768079A1E720E7D7E5799740D2798C
:02AD2E00AAE792
:10AD3000FAE5792323B4C500400274C42437300EE9
:10AD400030F42437300D15F7BA0302FA0AC39AF526
:10AD5000B175B300EAF5B4C313F5B222101C06D2E4
:10AD60001C76C88081763274FF200E02749B02AC80
:10AD7000E6C313247E80CDD2B5C28EAE8DAA8DAF30
:10AD80008BAB8BE4F58DF58BD28E3014012278B627
:10AD9000BE0007EF24E24002800806E624EC5002E1
:10ADA0007614206705E624F64005E4FEFAFFFB7CF6
:10ADB000007D0A125BCF7C007D5E125CEF8F7EEE21
:10ADC0006003757EFFEAFC7A33125BE3EBF5F0A4D7
:10ADD000E5F0CB8CF0A425E0C5F035E0CB926C25F6
:10ADE000F050060BBB0002D26C30E7060BBB000232
:10ADF000D26CECF5F0A42BFBE5F03400FC306C01D8
:10AE00000C78A6E6C39BFF18E608F6EB18F618E6E2
:10AE10009CFE18E608F6EC18F6301401227A005071
:10AE2000040A125E667C007D6E125CEF8FF078A2E1
:10AE3000E6A4FBACF0125E05EBBA0002F404FAE4FF
:10AE4000F8FFEA30E70118E57960062075031FF482
:10AE5000042AF579EF38D27520E70860037579FF89
:10AE600002BB73C2750470F5E579F40460EFF579FF
:10AE700080EE120982E5BE78A2F624F65007E4F5CA
:10AE8000BEF61248EB12097D85BC2B85BD21E5BEBF
:10AE9000F54824F65008E4F5BEF5481248EBE5BF46
:10AEA000F54324F3503924F3403512097878A1A6EC
:10AEB000BCE5BF789DF61424FB50087403F6F5BF7B
:10AEC0001248EB78B7A6BE12096EE5BDA2E3926602
:10AED000A2E49267035403C253B40102D253227412
:0AAEE0000DF5BFF5431248EB80C0EA
:10005E0078FFE4F6D8FDF478D8F6F5A6D220D2B41F
:10006E00D2C075C07A75D75075AE1375AF01758154
:10007E00D87590F875EFBC75FDFFD2A412D06FC283
:10008E00A4745012259B758951D28C75A882D2BC4E
:10009E0012AEEA12D16812B82312AE72C22012CB7F
:1000AE00DA1224667F527E019090EB126C09124890
:1000BE004412CFDC12D06F12CDBE12CFDC12D0980C
:1000CE007C1412D079300003022588DCF512438DA2
:1000DE00753A001243DFE53A701612D19C7F437ECB
:1000EE0006909754126C0912CFDC3000FD02258861
:1000FE0075A6FF12438D12AE72C22B12246612CF5A
:10010E00DC12D06B12D09878B5761E12CBDA12B8FC
:10011E0018C215C21412246690910A7F78126BF7DA
:10012E00205E0A7F767E1290911712C74D7F401285
:10013E00CFB87F497E0978AEE612C5B77E15743A00
:10014E0012C71F7E1AE53E12C5B77E26743A12C735
:10015E001F7E2BE53F20E00805A6E5A6700215A63A
:10016E00E53F12C5B77F5312BD897F577E0B12C470
:10017E00E412C56C7F6030737F7E0BAC5DAB5C129E
:10018E00C4E812C56C7E31126C947F697E1212CA5D
:10019E0075E5A60303543FFDFE0D7F7312D0E10FEC
:1001AE0012D0E11EDDF478B5E57124F64002761E1C
:0401BE00307419E69A
:1001C20060567F727E16744012C6ED7E17E612C626
:1001D200757E1F745312C6ED12CFDC10003710016A
:1001E2003710023712432BD2AC75369612CEEBB4CF
:1001F200E005124429800AE53670F112437B12D0E1
:10020200680201192074097E2BE52E540712C70CCF
:100212007E1702019502258802278B8078E5352416
:10022200C8504FE59020E24AD0E0D0E012027502B9
:1002320057D8E53524D2503AE59020E235D0E0D0C7
:10024200E012D19C803EE53524D25026E59020E292
:1002520021D0E0D0E012D19C306B1190935F7F09E6
:10026200126BF712CFDC12492712707B1202750251
:10027200047E2212D19C9097D37F00126BF712CF8B
:10028200DC02D06812D19C9097D37F00126BF712D8
:10029200CFDC12D06BC215C214C227C26812D0982A
:1002A2007537019091AF12179D9002AF7302010151
:1002B20002127802066502199402047E0204BB024D
:1002C20057D80202C712D0987537079094FC1217BC
:1002D2009D9002D7730202970204F60205300205CE
:1002E200610202FB02036D0202C70202C702033768
:1002F20002031E0246A50203001243E280481218BE
:10030200F512CFDC1000BE10010280F890935F7FDF
:1003120063126BF712CFDC12AF5380A91218F512D9
:10032200CFDC1000A010010280F812487012CBDA64
:1003320012AE7280907F49A25E12082E925E12085F
:060342004980821248EB25
:1003480012D0987537029096B912179D900358737A
:100358000202C70209AD020A12020A69020ABE02B3
:100368000B02020B1112D19C90914F7F017E091252
:100378006C099091577F0A7E09126C097F1312BD90
:1003880081751700120973E5BC12044DE5BD12040E
:100398004DE5BE12044DE5BF12044D9091977F5F65
:1003A8007E06126C0912192912CFDC751700120487
:1003B8002D10000810011510024880F20517E517E6
:1003C80024F7500375170075100080E2E5176408DC
:1003D800701512097375BC0175BD2375BE4575BFCF
:1003E800671248EB02036DE51012045F12CFDC12AE
:1003F800040D0510531007E51724FE40035310039E
:1004080080AC0202C7A9BCAABDABBEACBFE517133E
:1004180004F8E640085407C42510C4800454702525
:1004280010F60272637800E875F009A42417FF7EBD
:10043800347D20E8651770027D71ED12C71F08B87A
:1004480009E502CFDCF8C4120453E812045F7E0306
:100458000517E51702C70C540775F007A490915FBC
:100468002582F58250020583E51775F009A4241743
:10047800FF7E0C026C09C26812D0987537059092FD
:10048800DB12179D90049073020297026E48026E69
:100498008D02701C02047E0204B4026F5E026FC4F7
:1004A80002124102047E0212270207717F2E1211E6
:1004B8003280C312D0987537069093A212179D9078
:1004C80004CB7302029702127E0212E00213570253
:1004D80014240214560214CD0204BB0204EC0215C3
:1004E800000215A57F4912113280C81248EB12D0BC
:1004F8009875370390956612179D9005067302024A
:10050800C7020792020DFC0207A70207B202119C5C
:10051800020E83020855020EB7020EF10211EE0216
:100528000E6B020F3F1248EB12D098753704909665
:100538002A12179D900540730202C70207C10207DD
:10054800CC0205300207E20207ED020B2B02053050
:100558000207FC0207D71248EB12D09875370B90A8
:10056800966F12179D900571730202C7020BCA029B
:100578000BCA0205980205D502056102056102123F
:1005880084020C56020D23020CC9020DB202081691
:100598007F1C1209A512096EA8BE1205C912CFDC6C
:1005A80010000810010D10021480EF18B800EB7845
:1005B8000B80E708E824F450E1780180DD88BE80EC
:1005C800957F1B7E35E875F005A402C5B77F251217
:1005D80009A512096EA8BF12060712CFDC10000881
:1005E80010010D10021480EF18B800EB780980E7AD
:1005F80008E824F650E1780180DD88BF02055E7FB7
:10060800247E3BE802C70C120991E5BF541F75F020
:0D0618003CA4ACF0FDE5BE75F005A42DFD81
:10062500E5F03CFC12096EE5BF1475F005A485BE26
:10063500F0A42DFFE5F03CFE7C007D3C125CFCC087
:1006450005EF75F01884E5F07F2D7E2412C5B77E81
:1006550030743A12C71F7E35D0E012C5B702CFDC21
:10066500D25712D19C12188C1206730202977F176B
:100675007E02909201126C097F4C7E0290921812B4
:100685006C09AC5DAB5C7F577E0412C564120991A1
:1006950085BC6285BD63E56124F840449092237F63
:1006A50037126BF7AE61AF607C017D5E125CFCC3F7
:1006B500741F9FFAAC63AB62EC3392175003125E62
:1006C50076125BE3AB047C00301703125E7674F59B
:1006D5002BFB74033CFC125BB97F377E1512C4DC1F
:1006E5009092307F697E0F126C09E560240FFBE460
:1006F5003561FCA25C923BD25C7E1E12C4E8A23B33
:10070500925C7E30742012C71F7E36742012C71F7C
:10071500E5602562FBE5613563FC7F227E0412C539
:1007250064E56245637016742E7E3A12C71F12CFB8
:10073500DC10000D10011510022602069B742080A6
:10074500E81562E562B4FF0C156380080562E56291
:1007550070020563E53524F5500375330102069BE8
:100765001209918562BC8563BD0248EB1218F5122A
:10077500CFDC10001510010280F87F637E05909391
:100785005F126C0912CFDC1248F602047E1209785A
:10079500E5BCA2E77F0A120837E5BC92E7F5BC0283
:1007A50004F37F1CA20D12082E920D80097F25A24D
:1007B5000E12082E920E1208490204F67F0AA20FA5
:1007C50012082E920F802A7F13A20812082E920873
:1007D500801F7F52A20C12082E920C80147F25A236
:1007E5000B12082E920B80097F2DA20912082E925A
:1007F500091208490205307F4912096EE5BDA2E3D9
:1008050012082E12096EE5BD92E39266F5BD02054A
:100815002D7F6D12096EE5BDA2E012082E12096E3C
:10082500E5BD92E0F5BD02055E12097D85BC2B850F
:10083500BD218F1F92171209A5AF1F1F7E39127890
:10084500CFA2172212097D852BBC8521BD0248EB5D
:1008550020371412097885BE12120882120978858C
:1008650012BE1248EB80057F3F1208740204F67E23
:10087500039095F2126C0912CFDC02D06875A6FFC1
:1008850012D19C12A969740712D1888FF0740612CF
:10089500D188EF2512C395F0FD78D8E6C4540F2D05
:1008A500A2E7923D4010FD24CD50027D32AC05C338
:0B08B500743F9DFD800FF404FD24C87B
:1008C00050027D37AC0574402DFD7F4012BD817E06
:1008D0001212D0E10EBE1EF91F303D020F0FEF6D58
:1008E00070EDE536700A753606EC2513F5148C1399
:1008F00012090912CFDC100007100108300207228C
:100900001512800205120208827F377E28742E128B
:10091000C71F7F347E21740A303D010412C73CE5B5
:1009200014FC249C50027C63EC75F00A84C0F07FB8
:10093000347E2D12C73CD0E07F377E3612C70C7F45
:10094000437E1E12C4E47E00E51212C67B7F057E44
:10095000029095FE126C097F6D7E01909609126CD3
:100960003C7F747E0490961B126C3C02188C75C6FA
:10097000F6802B75C6F7802675C6F8802175C6F9F6
:10098000801C75C6FA801775C6FB801275C6FC8080
:100990000D75C6FE800875C6FF800375C6FD75C758
:1009A0000375B90122743F12C6ED02CFDC7F0A1233
:1009B00009A57E2A1243E2120982A8BF1209E1109A
:1009C000001210010510021580F508E824E750EC2C
:1009D000781880E818E830E7E3780080DF88BF8087
:1009E000627F097E0590984BB80C03909845126C75
:1009F000097E27E53D28240C75F01884E5F012C522
:0F0A0000B77E33743B12C71F7E35E53E12C5B774
:100A0F0002CFDC7F131209A512097D85BC2B120AB8
:100A1F004610000810010510021780F2105C072025
:100A2F005D0BD25C80E8105DE5D25D80E1D25C8029
:100A3F00DD852BBC020345205C10205D1890989E2D
:100A4F007F127E23126C0902CFDC9098B2205DF0EA
:100A5F009098A580EB9098AB80E67F1C1209A512A9
:100A6F00097DA8BF120AA010000810011110021A68
:100A7F0080F2E824F250031880EA780D80E6E8242B
:100A8F00E740030880DE781980DAE8F5BFF5438088
:100A9F00A37F1B7E26E412C70CE82323B464087ED1
:100AAF0026740112C70CE47E2E12C5B702CFDC7F6D
:100ABF00251209A512098CA8BCE8120AF912CFDC7D
:100ACF0010000810010D10021F80EEE824E050E91D
:100ADF00188006E824CF40E10812098C88BC124820
:100AEF00EBD21512CBDA80D180157F247E3724E22A
:100AFF0002C6287F2EA20A12082E920A1208490255
:100B0F0003487F3712096EE5BDA2E412082E1209C1
:100B1F006EE5BD92E49267F5BD0203457F367E1503
:100B2F00743E12C71F120978A8BD120B9512CFDCA5
:100B3F0010000810010510021080EFE82487500400
:100B4F00240A800224E8F880E17F367E29743E1261
:080B5F00C71F120B9512CFDC39
:100B670010000810011410022080EF18B80904784B
:100B77007880E7B878E478E780E008B87904780AFD
:100B870080D8B8E8D5787980D188BD02052DE824CA
:100B970087923DE8500224917F367E2FC313923B04
:100BA70012C6287E3CE4303B02740512C7057E1A44
:100BB7009099D9303D039099DD126C097F3C7E3ABC
:100BC70002D0E17F127E1F743E12C71F120991A83F
:100BD700BF53001F53BFE0120C3910000810010D5E
:100BE70010021480F218B8FFEE781780EA08E8249C
:100BF700E850E4780080E0120C397E2F743E12C76B
:100C07001F12CFDC10000810011110021B80E8151D
:100C1700BEE5BEB4FFE175BE0B80DC05BEE5BE24B4
:100C2700F450D475BE0080CFE8541F25BFF5BF022E
:100C3700055E7F127E24E812C5B77E30743A12C76C
:100C47001F7E35E5BE75F005A412C5B702CFDC7F60
:100C5700491209A5120C8CF853BF1F120C961000ED
:100C67000810010D10021280F218B8FF02780480F4
:100C7700EA08B80502780080E2E8C42354E025BFFB
:100C8700F5BF02055E120991E5BF54E0C403227F58
:100C9700487E059099F3126C09E8601CB4040A7E3B
:0F0CA700059099E8126C09800C9099FF126C0966
:100CB6007E38E812C70C02CFDC9099FA7E29126CB6
:100CC6000980F3120C8C60206404601C7F5B12099F
:100CD600A512097D85BC2B120CFE12097D10000B96
:100CE60010010810020C80EF020561105FE9D25F67
:100CF60080E5852BBC02055E120C8C601F640460C7
:100D06001B7F5A7E059099F3126C097E23909A03F5
:100D1600305F03909A0A126C0912CFDC22120C8CF7
:100D260070030205307F521209A5120982A8BC126F
:100D36000D6112098210000810010810020880EFE8
:100D46001880EC0880E912098288BC1248EB120967
:100D56008CE875F005A4F5BD02055E120C8C604B9F
:100D6600E875F03270040475F028A4ADF0FC305D2F
:100D760011ACF0FB7A8A125BF1EB30E7050CBC0094
:100D8600010DAE05AF047C007D64125CFCC005EF6E
:100D96007F517E1A12C5D47E2C742C12C71FD0E048
:100DA6007E2F12C5B7123CD112CFDC227F64120906
:100DB600A5120982A8BD120DDF10000810010D1042
:100DC600021280F218B8FFEE787D80EA08B87EE657
:100DD600780080E288BD02055E7F63E82312C125A4
:100DE60075F06484C0F07E2612C70C7E2C742C121B
:100DF600C71FD0E080AA7F131209A5120978E5BCA7
:080E0600A2E7923DC2E7F8E803
:100E0E00120E3B12CFDC10000810010D10021280E2
:100E1E00EE18B800EA783280E608B833E27801803E
:100E2E00DEE8A23D92E7F5BC79A1F78079547F30D8
:100E3E005C01237F127E2375F00A84C0F012C6284F
:100E4E007E2D742C12C71FD0E07E2F12C7050F7E89
:100E5E00359098B8305C03909914026C3C7F641204
:100E6E0009A5120982E5BE7F637E2C127924F5BE98
:100E7E0079A2F780317F371209A512097DA8BC53DC
:100E8E0000037F367E32E812C70C12CFDC1000084A
:100E9E0010010710020780E718180880E2E5BC541D
:100EAE00FC48F5BCF52B0204F37F491209A5120983
:100EBE008CA8BE120EE612CFDC10000810010D1029
:100ECE00021280EF08B800EB789B80E718B89AE31F
:100EDE0078FF80DF88BE80CEE8F424647F487E2CC5
:100EEE0002C5D47F521209A512098CA8BF120F2079
:100EFE0012CFDC10000810010D10021280EF18B88E
:100F0E0069EB788F80E708B890E3786A80DF88BF56
:100F1E008094C3E89435F5F0A4AEF0FF7C007D39E3
:100F2E00125CFCEF7F517E2C12C62E7E3BE402C774
:100F3E00051226CD754A00D210C211D214D2757583
:0A0F4E00791475340012D19C7F0065
:100F58007E029095D3126C09903CFA7F087E261287
:100F6800C74DE52B54030F7E3912C70C1218A71270
:100F7800C3B512833512CFDC10000810011A100215
:100F88002480C5207504057980BE1579E579B4FFFC
:100F980005C27575790180B02075EB1579E5797012
:100FA800A7D27580A3C210C2140204F612097DE507
:100FB800BE7F097E3A02C70C120982A8BF1209E156
:100FC80012097D85BC2B85BD21120A46A8BF120ACD
:100FD800A012098CE5BC120AF97F2DA20A1210E7AB
:100FE8007F36A2670210E712097D85BC2B85BD21DB
:100FF8007F1BA20D1210E77F24A20E1210E7120920
:1010080078E5BC120E3B7F09E5BCA2E71210E7A801
:10101800BF1211DAE52B54037F367E3212C70C1249
:101028000982E5BE7F637E2C12C70C12098CA8BE0C
:10103800120EE6A8BF120F2012096EA8BC02121FDA
:1010480012097D85BC2B85BD217F09A20F1210E7EF
:101058007F12A2081210E712096EE5BDA2E37F48CD
:101068001210E77F51A20C1210E77F24A20B121076
:10107800E77F2DA2091210E7120978A8BD020B9587
:10108800120991A8BF53001F120C3912096EA8BE8D
:101098001205C9A8BF12060712060F12097DE5BE80
:1010A8007F3F7E3A12C70C120991E5BF54E0C40392
:1010B800F8120C96120982A8BC120D6112097D1251
:0210C8000CFE1C
:1010CA00120982A8BD120DDF12096EE5BDA2E07FEA
:1010DA006C800A12097D85BC2B7F48A25E744E4043
:1010EA000274597E3A02C71F12726F7F73126F0B16
:1010FA001272BE7F6C126F1A7F2D800E12097DE567
:10110A00BE7F097E3A12C70C7F4812096EE5BD03FD
:10111A005403F51075F005A47E1E9093732582F58D
:10112A008250020583026C091209A51F121114A824
:10113A001012111412CFDC10000810010810022737
:10114A0080EF18800108530003202B03530001C2CB
:10115A0053B80102D253E8235406F9E5BD54F929DC
:10116A00F5BD1248EB80CA22125A4EEBF516F51459
:10117A007F6C126F1A125A327F647E23E51612C6EA
:10118A008BC3E5169514F5167F73126F0B7F2D022C
:10119A0011147F2E1209A5120978A8BFE824FA4073
:1011AA000330370278031211DA12CFDC100008106C
:1011BA00010D10021280E518B800E1780580DD08FB
:1011CA00B806D9780180D5799DE8F7F5BF0204F30E
:1011DA007F2D7E2C7420B80502742E12C71F7E3212
:1011EA00E802C70C7F5B1209A512096EA8BCE812B7
:1011FA00121F12CFDC10000810010D10021280EE2F
:10120A0018B800EA780380E608B804E2780180DEBC
:10121A0088BC0204F37F5A7E2CE802C70CD2687598
:10122A00480A1243E2D2141225D01273A9122F1CB3
:10123A00C26B12024880F3D2147515011272297515
:10124A00B901E5BC20E71C12735975A6FF1273B5E4
:10125A001218B212CFDC126D1210000F5005126E66
:10126A003A80E70515E515242050D102047E1212B2
:10127A008A02029712128A0204BB12128A020561BA
:10128A0012129612097D8548BE0248EB1225C21237
:10129A0025DC12628912D19C909405D249127C01F4
:1012AA00127BBA12186212CFDC100014100105105A
:1012BA00021B80F50548E548640A7002F54880CFAC
:1012CA001548E54864FF700375480980C285484996
:1012DA001225DCE558221243E21225C2854849C28A
:1012EA0050E558B40F02D2501262898038D227755D
:1012FA00480A1225D012628912D19C127B29909732
:10130A009A2029039097A5121916C26A122F1C1047
:10131A006A0280E1C2271272018549481216D41264
:10132A0025DC12628912D19C909342127BFF2050D5
:10133A000E12190012CFDC1000101001B080F81242
:10134A0018B212CFDC10000280FB0204BB1225C2C5
:10135A00E55830E7137F1B9097847E05126C0912BB
:10136A00CFDC12D06B0204BB1225DC1262898559CC
:10137A004912D19C12189C9097A5127BFF127BC42C
:10138A0012CFDC10000810010A10020C80F51213AB
:10139A00EF80DB1213FC80D612D19C12189C909419
:0113AA00152D
:1013AB00127BFF127BC4127BC812CFDC100008101B
:1013BB00010A10020C80F512140880DB121416803F
:1013CB00D612169A1225DC12628912D19C909707BD
:1013DB00127BFF1218DA12CFDC1000051002888086
:1013EB00F80204BB0559C3E55895595003755900CC
:1013FB00221559E55964FF7003855859220549D3C5
:10140B00E5491495584003754900221549E549648F
:10141B00FF70058558490549221225C2E55830E76A
:10142B00057F240213611225DC12628912D19C9074
:10143B009420127BFF12190B12CFDC10000A100143
:10144B000280F812174380DE0204BB1225C2E55856
:10145B0030E7057F2D021361C26B7559FF1262894C
:10146B0012D19C12188CE55930E7031218A79094EF
:10147B0031127BFF127BD412CFDCE55820E706102C
:10148B00000810011110021B80F00559C39559502B
:10149B00CF7559FF80CA1559E55964FE70C285583E
:1014AB005980BDE55920E711D26B75A700758307ED
:1014BB00C4F582E0B2E7F080A7306B031216F1029D
:1014CB0004BB1225C2E55830E7057F3602136112C3
:1014DB0025DC12628912D19C90943C127BFF12186E
:1014EB00F512CFDC10000B10010280F81217381226
:1014FB00176D0204BB1225C2E55820E7087F5190F7
:10150B00944602136412D19C9097B0127BFF121871
:09151B00B212CFDC12431BD2AC6A
:1015240010001FE55830E7F8306DF512163A7E20AA
:101534007F0050139097C9126C3C12CFDC12D06B11
:1015440080CAC2AC0204BB1B8B1390935F126C3C29
:1015540012CFDCC26B7B007514B812172D127328DE
:101564001272DA5025A814E824384004A6010514A0
:101574000BC3E5139B50E678B812176F306B031258
:10158400707B1225DC126289808212726FE516600C
:10159400E6D26B127385C003127240D003A9158082
:1015A400C41225C2E55830E7057F5A02136112259B
:1015B400DC12628912D19C909451127BFF1218CFD5
:1015C40012CFDC10003510010280F87546051216A2
:1015D4000250157F007E357407954612C68B12CFD4
:1015E400DC12D06BD546E7D39097BB50039097C9D4
:1015F400127BFF12CFDC12D06B80B30204BB124308
:101604001B12CD86745212CDB9745412CD54E558C0
:101614000475590012CD75126CC140161272011274
:101624007359126D12400B0559C3E558955950EC86
:10163400C322C2ACD32212431BD2AC12CEE6204C3E
:10164400F1B440F712CEEBB4400312CEEBB452E245
:10165400F53812CEEBB454DA12CEEBFA60D424EFA0
:1016640040D012CEEBE53870C912CEEB12CEEB129D
:101674006CA67B007E03126D9D50102050B412CED8
:0E168400EB204C03B440F7DEED80A712733864
:101692000B126CA6DAE0C32212177EE55924C8F8B1
:1016A2008602E54924C8F9986013146010500F1897
:1016B200E608F618E86970F7A70212176D22E559D5
:1016C200640F60F91908E618F608E86970F7A702CE
:1016D20080E812177E78C8C250E6B4FF028007087D
:1016E200B8D8F6D25022B8D702D250A615807C784C
:1016F200B8121780E4F9F5A7758307E9C4F582E00B
:1017020030E70AE924B8F82438400276FF09C3E535
:10171200589950E712173878B879C8E6B4FF0280B2
:1017220002F70908E8243850F2804079B877FF09B7
:10173200E9243850F82279C877FF09E9242850F8BB
:101742002212177EC23D78D7B6FF04A900D23D18F7
:10175200B8C7F5203D0279D81978C8B6FF0122C36F
:10176200E8995007C6C7C6081980F478C812178FBF
:1017720012739712739712739702739778C812179E
:101782008F12737312737312737302737375C703B9
:0E179200E54875F004A42480F5C62212D19C0F
:1017A000C23C126BFBE537604E1460481460401475
:1017B000603814603014602814602014600E1460C7
:1017C0000B14600D14600514600C802B1210DD806A
:1017D000261211728021121088801C1211068017A7
:1017E0001210F28012121048800D120FEF800812B2
:1017F0000FC08003120FB412CFDC12D06F12188CFE
:1018000012AD05A81F08E814C23BB51D02D23B75F6
:10181000F007203C0375F009A4FF7E00303C0C74F7
:1018200020303B02743E12C6ED800A740B303B023E
:10183000740A12C705D8CF12CFDCE51D10000810BE
:10184000011010021880B9651F7003751DFF051D7A
:1018500080AE7005851F1D80A7151D80A375F00340
:10186000A4227F7B7E0090996C126C3CE54824F6A4
:1018700040087E0A909766126C3C22126F377E05F4
:10188000745B12C6E97E1D745C02C6E912187B7E89
:101890003490997D026C3C126F37800312187B7E66
:1018A00031909981026C3C12187B7E319097D40262
:1018B0006C3C126F377E008005126F377E2D90973B
:1018C000D4026C3C1218CF7E31909387026C3C128C
:1018D00018B27E1A90938C026C3C1218B280C0121F
:1018E00018B27E1890934C026C3C1218B27E1A907B
:0A18F00097D9026C3C1218B27E1A60
:1018FA009097DE026C3C1218B27E1A90940F026C1A
:10190A003C1218B27E1890942B026C3C7F007E2009
:10191A00126C3C02CFDC126F379097E4026C3A12D9
:10192A006F379097F5026C3A12B19112099BE5BD97
:10193A00F55EF56CE5BCF55FF56B756A007561FFE0
:10194A0075A70490070012B13DB4FC12E582C313D7
:10195A00F561E56CF0E56BF0E58260168005B4FF91
:10196A0002800F12B08CE56C655E70DAE56B655F1C
:10197A0070D475A70022E560758307C333F582E04A
:10198A00A3F56CE0F56B756A0022D214C21F121916
:10199A0032756000E561B4FF1612D19C9092337FD4
:1019AA000A7E05126C3C12CFDC12D068020297C282
:1019BA0010C21112D19C12188C301F0A7F07909204
:1019CA0041126C3A80647F007E01C3E56012C68BC7
:1019DA007E0E742812C6E98560487407F51FFF7EDB
:1019EA0000743E12C6EDE54812198212BB8F121F0F
:1019FA001B0548C3E5619548FD401CE51F2407F512
:101A0A001F24C850E17F387E01ED0412C68B7E0E7A
:101A1A00742912C6E9800DE51F2407FF7E019097FD
:101A2A00D3126C3C201F03121F5E12CFDC10001968
:101A3A0010012C10020280F5120234301F3D0202FE
:0B1A4A0086101F02D21F0219B9E561CF
:101A550060F4E56065617005201FF080E9201FE6F0
:101A6500056080E7E56160DEE56065617005201F62
:101A7500D58009201FD5E560700280CA156080CB2E
:101A850012193212198012BB8F122052756A101268
:101A9500B124122109909248D23C126BFB1217FD1A
:101AA500901AA9730219B9022D73021AD2021AB536
:101AB5001218F512CFDC1000C710010280F81219B8
:101AC5008012B13DC2E2FF12AF39021994C253121E
:101AD500198012BB8F75370090926112179D901A6D
:101AE500E773021A85021CD4021CD9021AD2021B02
:101AF5000E021B13021AD2021B51021B55021B595F
:101B0500021B60021B64021B6812434880031243D8
:101B150033780A121C31740712CD52121C7012CD83
:101B25006E121CAB12B12412B15012B04D12B26735
:101B3500121DC5D5150C75150A121CBE121EE5120F
:101B4500CD6E100204E57F70DB021A85780A8006E7
:101B5500780480027801124348800D780A8006785F
:101B65000480027801124333121C31740712CD47E9
:101B7500121C70E54812CD33742A12CD5412CD547F
:101B850012CD5412CD6E121CAB12B12412B15012EB
:101B9500B04D12B267121DC5D51548854815121CE2
:101BA500BEE51C12CD33E51B12CD33E51B2548F5EB
:101BB5001BE4351CF51CE4A27792E7A27492E0A21F
:0E1BC5007392E112CD33AD75AC74AB73E57D58
:101BD300C4121BF2AD78AC77AB76E57D121BF21223
:101BE3001F0312CD6E100204E57F709F021A855405
:101BF3000F2375F00584F8C3EB33FBEC33FCED33B3
:101C0300FDC3EB33FBEC33FCED33FD20E713EB2893
:101C1300FBE43CFCE43D12CD33EC12CD33EB02CDBF
:101C230033C3EB98FBEC9400FCED940080E8884808
:101C33001218B9E4F54AF549756A2075150112B110
:101C43002412B04DD5150E854815E5492401F549F3
:101C5300E4354AF54AE57F70E5744012CDB97478EE
:101C630012CD54746312CD54741F02CD47121EC09B
:101C7300E56012CD3312198012BB8FE53A12CD47BE
:101C8300E53B12CD47E53C12CD47E53D12CD47E597
:101C93003E12CD47E53F12CD47740112CD33E54ADD
:101CA30012CD33E54902CD33121980756A20E4F56C
:101CB3001CF51BF514F51375150122753800E51491
:101CC30012CD33E51312CD330513E513700205145A
:101CD30022124348800312431E1218B9121E1B120C
:101CE300D073756A2075150175A6FF754A0112B088
:101CF300C812B04D12B267121DC5D5150975151E50
:091D0300121DE912D07D121EE54B
:101D0C00E57912CD33E57EB47F01E4C33350027420
:101D1C00FF12CD33E571121DAA12CD33E57012CD31
:101D2C0033E57B24ACFFE55F340912CD39EF12CDDE
:101D3C0033E51520E033857D56E412CD33E52EC412
:101D4C0012CD3912CD7D12D07D10021A30559074FF
:101D5C004012CD54744512CD54744F12CD54744668
:101D6C0012CD5412CD7D021A85E556121D84C4FA8B
:101D7C00E57D121D842A80C2FBC4121D912323CB46
:101D8C00121D912B22540FFC24F650027C00901D46
:101D9C00A0EC932200000101010202030303FA24C8
:101DAC0040400A24804003EA3322D2E72274FF2207
:101DBC0020E703C3132224C022E53F701F7F7B7EE4
:101DCC000078AEE612C675EE2404FE743A12C6ED27
:101DDC00EE2404FEE53E12C66F12CFDC22C015D2F3
:101DEC0012129A42C212D01578AEE612CD47E53ED9
:101DFC0012CD47E53F12CD47E54512CD33E55212E2
:101E0C00CD33740A12CD3374C012CD3302CD7D7430
:101E1C004012CD54745412CDB9744E12CD54E412F8
:101E2C00CD33121EC0741F12CD47E53D12CD47E5D0
:101E3C006012CD3312198012BB8F78ABE60812CD2D
:011E4C00474E
:101E4D00E60812CD47E60812CD47E612CD47E53E2E
:101E5D0012CD4712244DE51212CD47E51112CD4793
:101E6D00740112CD33909806121F0D756A1012B1C0
:101E7D0024057F057F787F12CD2C787B12CD2C78B1
:101E8D007D12CD2C787712CD2CE4FEFF780712CD84
:101E9D002C12CD2CE57412CD33E57512CD33E41231
:101EAD00CD33E573C333500274FF12CD3312CD2CF5
:101EBD0002CD7D75C70375C6FF75B901C217751DB6
:101ECD000085BC1C85BD1B85BE1A85BF19125B69BB
:101EDD00EE12CD33EF02CD33E57512CD33E574122D
:101EED00CD33E57312CD33E57812CD33E57712CDD1
:101EFD0033E57612CD33E55E12CD33E57A02CD337F
:101F0D0075A700E493700122A312CD5480F5AF1F85
:101F1D007E0478ADE612C66F7E0C742C12C6ED7E73
:101F2D000E18E612C66F7E1A78AEE612C66F7E22C6
:101F3D00743B12C6ED7E24E53E12C66F7E2FE54042
:101F4D0012C6757E37743B12C6ED0E0EE54102C604
:101F5D006F75320012198012BB8F857946787A79A8
:101F6D006412BBA87464125F448E47122052756AC6
:101F7D0020D23D12B12412B150122089303D0930CA
:101F8D007406C23D8E1E8F1FE57F602BE54C24FF2E
:081F9D00F54CE54D34FFF54D54
:101FA500454C600512B06280D2751D3C12B12412F9
:101FB500B15012B04D122089E57F6003D51DED1299
:101FC50020EA90210212C74D203D0DAE1EAF1F1213
:101FD50020EA9020FB12C74DE546FD700B90993C19
:101FE500305D11909938800C047010909938305DEF
:101FF500039099347F38123CCB804BE4FFFC7E057F
:10200500305D047E027FB3125CEFAC06AB07125B5A
:10201500B97F38C23DE51C6007D23D7E2C12C6DA79
:10202500E51B203D026007D23D7E3012C6DAE51A77
:10203500203D026007D23D7E3412C6DAE5197E38AE
:1020450012C6DA123CD0E53224C850FA22E54075B2
:10205500F03CA42541FFF54CE435F0FEF54D7C0040
:102065007D10125CFC0F8F4BAF4CAE4D7C007D3C60
:10207500125BCF7C00AD4B125CFCEE4F70010F8FF5
:102085004C8E4D2278647973C2D11220A0FF7867F7
:102095007976D2D11220A0FE02D0E1C3E796FB08E3
:1020A50009E796FC0809E796FDA2E7921750031287
:1020B5005E7E75135A30D10E751320B217AA4712DA
:1020C5005C03AB04AC05E546600B04600BAA461245
:0520D5005C1AEB03FBA7
:1020DA00EB03FBEB543FFBE5132B2017029B9B22E0
:1020EA00EE141430E701E4FEEF141430E701E4FFC4
:1020FA002205057088A8887005052020F82020751B
:10210A00320012D19C7E1E7F1C12D0E1DFFB12D05E
:10211A00E17E1E7F1C12D0E1DEFB7E1D7F1D12D0E8
:10212A00E1DEFB7F007E2178ADE612C66F7E297460
:10213A002E12C6ED7E2D18E612C66F7E35742E124B
:10214A00C6ED7E3918E612C66F7F077E21745412D7
:10215A00C6ED7E25744F12C6ED7E2D78AEE612C608
:10216A006F7E35743A12C6ED7E39E53E12C66F7837
:10217A00AE12244D7F0E7E21744C12C6ED7E25745C
:10218A004112C6ED7E2DE51212C66F7E35743A12E3
:10219A00C6ED7E39E51112C66F7F157E257444128D
:1021AA00C6ED7E2DE54012C6757E35743A12C6ED2F
:1021BA007E39E54112C66F7F1C7E2F85715412C18C
:1021CA00F47F217E01909907126C3C7E0EAC77ABAE
:1021DA007612C5217E2B85795F85787B12CACE7FE0
:1021EA00287E0190990B126C3C751D2B751E10E50B
:1021FA00741224017E25742F12C6ED751D2D751ECD
:10220A002BE5751224017F2F7E029098FF126C3CF9
:10221A00E57360031222AE7F367E029098F7126C45
:03222A003CE5721E
:10222D001222AE122346121980756A209004E6E53B
:10223D006CF09004E7E56BF0AE4DAF4C7C007D404B
:10224D00125CFCBF00010F0FAC07AD07E4FED23DE1
:10225D0012B12412B1501222EFE57F602CE54C240F
:10226D00FFF54CE54D34FFF54D454C600512B06260
:10227D0080DE751D3C0E12B12412B1501222F4E510
:10228D007F600612B04DD51DED1222C47F7812BDB0
:10229D00937F767E00743012C6EDE53224C850FA75
:1022AD00227E2112C12512C68B7E2F90990F305D93
:1022BD0003909914026C3C9004E6E0FD9004E7E075
:1022CD00FCC3E56A9420FBE56B9CFCE56C9DFD5021
:1022DD00032410FD125DEE9004E8EEF09004E9EF9A
:1022ED00F022DD03AD040E7F78E55E20E72AE57A66
:1022FD008549F0A4A9F0E57A854AF0A429F9E435D9
:10230D00F0FAE55E8549F0A429E435F02AFAE55E98
:10231D00854AF0A42ACF9FFF12D0E1103D18C3EFDC
:10232D009B50131BEF6B600E8F018B0712D0E11FBB
:10233D00EF6970F8AF01AB07229098BC305C039049
:05234D0098D5754A401F
:10235200754900AF76E577FE20E76B7005EF241034
:102362005064EF24A8EE34FD40119098C1305C0314
:102372009098D9754A1975499A8075EF2450EE34B0
:10238200FB40119098C6305C039098DE754A0C753C
:1023920049CD805CEF24A0EE34F640119098C9300C
:1023A2005C039098E3754A067549668043EF24F012
:1023B200EE34F140139098CC305C039098E8754A63
:1023C20004754944802A8028EF2490EE34E84011B5
:1023D2009098CF305C039098ED754A0275498F80D2
:1023E2000F9098D2305C039098F2754A0175499A21
:1023F2007F40126C3A7F4612BD937F5F02BD93AE5F
:102402001E75F064305C0375F03284C0F0F870041D
:10241200EE2404FEE51D12C6EDEE2404FEE860077C
:1024220012C6DAEE2404FED0E075F00A305C0375C1
:10243200F00584A8F012C6DAEE2404FE742C12C64B
:10244200ED0E0EE8305C012302C6DAE53E2541F5C9
:102452001124C45003F511D3E63540F51224E85097
:1024620002F5122212ACFFC21012D19C7F057E0926
:102472009090E2126C097F137E0890249A12C74D45
:102482007F2B7E0190250212C74D20370A7F277EBF
:072492002790257412C74DCD
:1024990022113007FE1FE001E101F80F00061B00C1
:1024A900F80C00180E007C10007006003C2000E0BB
:1024B90006003E4001E004001E8003C004001F0026
:1024C90003C004000F00078000000F800780000090
:1024D90017800F00000027C00F00000043C00F0045
:1024E900100083E00F00200301F00700C00F01F87E
:1024F9000383007F87FE01FC000E3E1800000300E5
:10250900000000180000030000000038000000006F
:102519000000003000000000000000FC761F0E1CC7
:102529006030ECFCBC3F172DF0F978613866264F16
:10253900619A706070C60E1EE330E06060C60C1CC4
:10254900C360C0E0618C0C18C7C0C0C0E18C1C39E5
:10255900C611C0C4C19C9931963180C8C1FF1E31D2
:10256900E7E180F0C0EE1C31C38180061630918806
:102579002892884924904927909248A0E3C8BCC270
:10258900AFD2C075C0107581D874FE12259BC2B434
:1025990080FCD2A6C2A512ACE412D06F02AD0575BB
:1025A900C703E54875F004A42480F5C6C23C75B993
:1025B90001E5BC047002D23C2212097DE5BEF54852
:1025C90024F65003754800753400753704C228D2C3
:1025D90029D22A75C703E54824E75003754800E561
:1025E9004875F004A42480F5C6751607751700C24E
:1025F9003C12261D12261D12261D12261D8517584E
:102609001558755900E548B40A09E5586005F4609C
:1026190002055922203C1D75B90105C6AABCABBDEE
:10262900ACBEADBFEA12263EEB12263EEC12263EA8
:10263900ED12263E22203C07F515B4FF03D23C22B9
:10264900C0C7C0C612722975A704851683E517C4C9
:10265900F8F58275B90105C6E5BCF0C582F824060E
:10266900F92403C582E5BDF0E5BEF0E5BFF075B913
:102679000105C6E5BCF0E5BDF0E5BFF08516838927
:1026890082E4F075B90105C685BC1385BD14E4F073
:10269900F08882E5BEF0E5BFF075B901E5BCF0E56B
:1026A900BDF0E5BEF0E5BFF0758306E51723541EBE
:0226B90024B04B
:1026BB00F582E513F0E514F075A700D0C6D0C70579
:1026CB00172212AE7278BEA64808E4F6F5590876C2
:1026DB001808F6D23608760A08F6060876BEC22522
:1026EB00C254C25512B1A61225D0C229C22AC207A2
:1026FB00C227C268C243C24AC246E4F52EF534F57E
:10270B0036F52F78A8F678B6F678B5F678A9F67878
:10271B009EF678B8A65E08A67A12C48AC26BC2333C
:10272B00C238C240C223C22212275B75460278C54B
:10273B00A646C23AD221C219C22685705778BA74FE
:10274B0001F608F608F608F6E4F542F541F54022E5
:10275B00E45407205E09B4040040027403801B128A
:10276B000973C313A9BC600C14A9BD600714A9BEDF
:10277B006002A9BFE94001C45407F53722020101E9
:10278B00754E501226CD1279F07544031243DF12A9
:10279B00A269D54403022588201EF1789F768075A7
:1027AB004A0012AF92D210C211C213C21212432BA3
:1027BB0075A60C12CBDA12B818E5A624FA4006124D
:1027CB00437B75A60C202517E59020E206E5352402
:0527DB0005400CE59033
:1027E00054057009E53524E25003022887E53224B8
:1027F00018400D75F00C84E5F070C9122F1F80C4CD
:10280000D21ED2AC306DBD7532F012CEF0B4E0B451
:10281000124429E53124F39205201203122CC3122D
:102820002841C01412827BD01412298E122F1F123D
:102830009A1112B39F122F1F1279F3122F1F022722
:10284000B830123AE54024F040257A0AC3E53F95B6
:102850004B601C402A24E24016E53F453E7003755C
:102860007E7F305405C254757F0112AFBEDADDE5BC
:10287000510404F57F24FE4003757F02C27722F4E1
:102880000424E250EA80D212D19C7F2A7E0E9098D6
:102890000A126C0975A6FFC2101012137F367E084B
:1028A00090936A126C0912CFDC12D068020101D237
:1028B0002112440312AFC87F1E7E0B90975E126CEC
:1028C0000912CFDC1228DA7F3E7E079094DA126C70
:1028D0000912CFDC12D062022588D215D22012B1A3
:1028E0007D12097D852BBC8521BD75B90575B902A1
:1028F00012B187D25512B0867F0012AF39D22012A2
:10290000B187E56A600512B04D80F7857A62D22002
:1029100012099B85BEBC85BFBD856BBE856CBF752E
:10292000B90575B90285BD6C85BC6B756A2012B19D
:102930007D122B3312B0BA12B187756A0012B1241E
:10294000E57064FE70437570FC854077854178853D
:042950001F7978185B
:10295400797A12BBA812AFF77FB412B0A6D22012B4
:10296400D07D12B187756A1012B1248554717F0825
:102974007810797212BBAA85627C855E7D12AFF7EE
:102984007FC412B0A6C220C21522300A012212430B
:1029940048122ADF745212CD54744D12CD5474432C
:1029A40012CD54122AEE12CD8F7441207402745643
:1029B40012CD54122A3B122A8512CD8FE53C12CD3A
:1029C40047E53B12CD47E53A12CD47122ABB12CD5B
:1029D4008F744512CD54122B24122ADF744712CD62
:1029E40054744712CD54744112CD54122AEE122A53
:1029F4003B12CD8FE43074010412CD5212CD8F906E
:102A040004C3E012CD4712CD8F9004E4E075F00AC0
:102A140084AFF012CD4712CD93EF12CD52AC5EAB22
:102A24007A122B00AC5DAB5C122B0012CD8F12CD51
:102A34008F122B2402432B7875C23D122A467878D4
:102A4400D23D12CD8F1276D5303D05E51E12CD5202
:102A5400E51D12CD52122AC8E51812CD52E57D208B
:102A64003D01C4540F12CD5212CD8F303D0974452F
:102A740030170274578007744E301702745302CD16
:102A840054207408122ABB122ABB802775A704900D
:102A940004BFE0FCE0FB7A1B125BF17832125D9319
:102AA400125BB9122AC59004C1E0FCE0FB125BB9C9
:0F2AB400122AC575A7002212CD8FE4F51AF51965
:102AC300800D12CD8FE51C12CD52E51B12CD52E5C0
:102AD3001A12CD5212CD93E51902CD52742412CDA0
:102AE30054744712CDB9745002CD5412CD8FE53DC5
:102AF30012CD47E53E12CD47E53F02CD4712773170
:102B030012CD8FE51D12CD54781CE612CD5218B8A4
:102B130017F812CD93E412CD5212CD8F744D02CD1E
:102B230054C038742A12CD54D03812CD6E02D07DE1
:102B330078107F0EE4F608DFFCF564F565F567F5BC
:102B4300687515FC751AC0751DC0756640756940BA
:102B5300754A0112B0C8305503022BF312B04DE58C
:102B630071B510004002F510E57EB47F01E4B511A4
:102B7300004002F511E512207502E513C395795063
:102B830006207545857913D3E57A9514E515648098
:102B9300FFE55E64809F400C857A14855E15857B16
:102BA30016855F173074A9C2D178647973122BD15B
:102BB30078677976122BD1D2D178187973122BD109
:102BC300781B7976122BD1808785791280B9D3E768
:102BD300960809E7960809E66480FFE764809F206A
:102BE300D101B3400AE7F61819E7F61819E7F622F8
:0E2BF300E51AB4C00E7873791812BBA8787377
:102C0100796412BBA878187964C2D1122C64741843
:102C1100125F448E47AE1EAF1F781B7967D2D11267
:102C21002C64C3E51F9FE51E9E50048E1E8F1F7EE0
:102C3100FF7FFFAC1EAD1F125CFC7A04EF8AF0A48B
:102C4100E5F0CE8AF0A42EFEE435F0BEFF011E6051
:102C5100051460057EFF8E1F22EE7E0020E7F77EC1
:102C6100FE80F3C3E697FB0809E697FC0809E6979F
:102C7100FD1818191930E703125E7EC3EB33FBEC24
:102C810033FCED33FDEB33EC33FBED33FC30D1059D
:102C9100AA47125C1A0BBB00010C751E03751FFFBE
:102CA100EC24FC40048C1E8B1FE627FB0809E63749
:102CB100FC0809E637A2E713F618EC13F618EB1334
:102CC100F62210131978B5E624FA401AE57124F6B4
:102CD1004008E57924F6400280380606803412D097
:0E2CE10079E59030E2DFD220753612D22EE473
:102CEF00F534F55A12B1D8122D19C219C25712273D
:102CFF005B1285BE1285EBD212853F4B754C0020BF
:102D0F005E02D228122745C22022D214122D68E665
:102D1F00F008DFFB857A62122D5E7570FE783A79C6
:102D2F007112BBA812AFF7122D5E85627A855E7B9A
:102D3F0012099185BC7E85BD7F7570C012AFF712E9
:102D4F002D68E0F608DFFB75A700D254C214227479
:102D5F00FF7870F608B880FB2275A7049004F0780E
:102D6F00707F102212198012BB8F12B2F49004EAF6
:102D7F00ECF09004EBEBF012431E751F03121E1BB9
:102D8F0012D079D51FF71226CD12D19C12CFDCC2EB
:102D9F0058C259756A2012B0C8125F428E47754AE1
:102DAF0001753901C210D211D214D21212B1D81238
:102DBF0085BE1285EB12CBDA75A6FF753609753213
:102DCF0000E59020E206E5352405400CE59054051A
:102DDF00701FE53524E25019C211C21212D19C1294
:102DEF00CFDCE4F535F52F7E0612D075C202021A3C
:102DFF0085E54A20E01612B2D712431E12CD867413
:102E0F004912CDB9780412CD2C12CD6EC221E54AEC
:102E1F00B40202D22112B0C8129A1130260F1262D8
:102E2F00EB1279F3753606E53670FCC2261279F08F
:102E3F00122F1FE54A20E022B4020A753900E53649
:092E4F0070F9022DC4E53960F9A7
:102E5800FD24E24002053912B0C82026C8DDF880FA
:102E6800E875390012431ED2ACE536602712CEEB66
:102E7800B440F612CEEBB4400312CEEBB44915F5CC
:102E88003812CF1BFC12CF1BFBAD3812CF1B6D7055
:102E980003122EA0C2AC80B1C39004E9E0FF9B905E
:102EA80004E8E0FE9C50048E048F038C148B137A84
:102EB80010125BF174202BF56A9004E7E03CF56B87
:102EC8009004E6E03D540FF56C754A0112B0C8AEA7
:102ED80014AF137C0E7D10125CFC8F40AE04AF055E
:102EE8007C007D3C125CFC8F418D429004EBE02518
:102EF80013FF9004EAE03514FE7C0E7D10125CFC92
:102F080078AEA607AE04AF057C007D3C125CFC8F52
:102F18003E8D3F2275370410003A10011610021634
:102F2800E52F5407600312ACF920783D20790A2078
:102F38007A1F2202310802306BE5376009146009F4
:102F4800146009023191023124023162C2790231DE
:102F5800AE02308FE53724FC500FE5376407600375
:102F68000232290231ED0230352011FAE59020E2D3
:102F7800028058753400201203D2132278A9E67013
:102F880019C226767DE5377005106B02D26BD277B1
:052F9800D24A75361459
:102F9D00D22E02B1CDE5376043146040B402272034
:102FAD000B24E6249B401F2414501C1285BE9097C1
:102FBD00317F207E08126C0912CFDC753608D22EB7
:102FCD0078A9E624ECF622241940FB241450F712BC
:102FDD0085BE1285EB90973A7F2980D72028E7E5AB
:102FED004824F640E1E5580460DC7F5D7E10E62460
:102FFD009B40D324145015C2330559C3E558955938
:10300D005005855859D22690971F80A9241940B68E
:10301D00241450B2E55960021559102606E5596081
:10302D00021559909728808D10780122753900E589
:10303D003424384007754A0175340022700AE54A78
:10304D0030E0F2754A0280F0146008754A06128568
:10305D00EB8006754A041285BE75390180DA302978
:10306D0009C229D22A7559008005302A0CD229129D
:10307D007BB0127B7E75340022206841302703D24D
:10308D006A22D2221233C512CFDC107A0122E53426
:10309D002438400712275B75340022700FAA3712AF
:1030AD00275B6A70F2740112275C80EB0412275CB7
:1030BD0024FC50E3E537B40706D22880DA8036C207
:1030CD0028E53724FC2324BEF879C4E7F9A748097D
:0230DD00A759F1
:1030DF0079C4E8F78648088607E537B405057548CB
:1030EF0018D2361225DC8F59E53764067002D207E5
:1030FF000230A41233A102334BE53760181460532A
:10310F0014600C14607CE53724F940060232A302E8
:10311F0031DC023270D223123BB610790122E53432
:10312F002438400775460175340022700EE5462499
:10313F00FE40F1E54660ED154680ECB40500500CFD
:10314F0004F54624FA50E075460580DB100FD8D2FF
:10315F000F80D4D223E53464C86003123BB61079D4
:10316F000122E534243750097011105B32D25B8095
:10317F002E100802D208123BB68024100C21D20C5C
:10318F00801DD223123BB610790122D24BE5342495
:10319F00374010C258C259201105D22E7536077507
:1031AF0034002224FD401524037006D258C25980E2
:1031BF00EEC258D2591460E7D25880E3120978E56D
:1031CF00BCB2E7F5BC79A1F71248EB80D278B8A66C
:1031DF005E08A67A2011C8753605D22E80C130122E
:1031EF002B127BEA055BE55B75F00B84E5F0F55B75
:1031FF00E55A24F64009E55A955B5003755B0012BA
:10320F007BEE12CFDCE5346003D534D27534002267
:02321F00D229B2
:10322100D22A75480A023311C2401007F13029032E
:10323100023311127BAC127BC0102A1BC233055919
:10324100C3E558955920E7025008755900E548B47F
:103251001816E558B4FF03755900127BD412CFDC60
:10326100E5346003D534C122D22A127BB080EE301E
:103271001223127BEA155BE55B30E70C755B0AE50F
:103281005A24F64003855A5B127BEE12CFDCE534FB
:103291006003D534DA75340022D229D22A75481751
:1032A100804CC2401007F2202944127BAC127BC033
:1032B100102A22C2331559E55930E71C855859E5C2
:1032C10058B4FF03755900E548B41802800AD22AA0
:1032D100127BB0800E855859E558B4FF037559002B
:1032E100127BD412CFDCE5346003D534B522201033
:1032F1006220115F7F180548E54864187008F54899
:1033010030270375480A1225A8303C2DDFE88026B6
:1033110020105A2011577F181548E54830E70575E8
:103321004817800A6409700630270375481712256B
:10333100A8303C05DFE275480A1225DC126289E5F6
:1033410032244C5005127B7E8003127B2975340098
:1033510002CFDC1233887F15E5486B70048A488000
:103361000205481225A8303CD0DFED80CC1233880D
:103371007F15E5486A70048B48800215481225A81C
:0D338100303CB6DFED80B27A007B09E53705
:10338E00B40401227A0A7B17B40601227418FAFBE0
:10339E00F5482275A704758307E559C4F582E0E068
:1033AE00F573E0F574E0F575E0F576E0F577E0F5A8
:1033BE007875A700026289E59020E23EE534243755
:1033CE0050381234091233E6205E4C7F2C90916DEA
:1033DE0012344D9091748067E534243775F009A44A
:1033EE002435FF205E0624BE50027F3EEF249B5004
:1033FE00027F627E26747112C71F227D077F3312F1
:10340E00341B0F12341BEF2408FFDDF3227E2F1224
:10341E00D111DEFB02D1117F2C120973E5BD1234DE
:10342E0036E5BE123436E5BFF8C412343CE8540714
:10343E0075F007A490915F2582F58250020583EF07
:06344E002409FF026BF7E8
:1079ED00027A9E12D19CE53724FC40F4B4FE14209B
:1079FD00110EE590F45407600122E532247450EF26
:107A0D0002828712D19C12C8C412C95612C13312F8
:107A1D00C1D312C4E012C3297E197F3612C27D1262
:107A2D00CE4512C293C206E537600514602D804A1B
:107A3D00C23A127B42123C72123D381240B01249CA
:107A4D007612499E123924E54864186009E54824E8
:107A5D00F6500312419B12D0B28011D23A127B68BC
:107A6D0012345C123CDD12BCE712D0CA12654C1206
:107A7D00C99D1260AC12635E800F127B4E12BC3535
:107A8D0012CA7112BCCB12D0A212821D12C2558025
:107A9D000C12D19CE53724F9401E127B2B302209A4
:107AAD001233C5E5347002C222302309123BB6E50C
:107ABD00347002C22302CFDC12188C75170012CC61
:107ACD00847F1212BD8130124A75100075A704759E
:107ADD008306126344E51075F009A42415FFF5170C
:107AED007E00E512602F75F06484E5F00F12C66F0D
:107AFD001F7E0EE51112C19175162312649E05109D
:107B0D00C3E55A95104006E51024F550BF30120319
:107B1D00127BEE8088745D12C71F80D5C249302953
:107B2D0005121862800312188C909342127C01206A
:107B3D002A71027BD4301223305E2030501D027E1C
:107B4D00DD301217305E06200B110284F412BD7A5F
:027B5D007F1790
:107B5F0012CFB875172002CC8412C83B12C7DC3085
:107B6F00120C20510302C89B12C0BF12BE9F22E409
:107B7F00FEFFE54824F6400D909766126C3C7E168A
:107B8F00E54802C6DAB40E0690976C026C3C9097EB
:107B9F0074126C3C7E12E54824F702C6757D208076
:107BAF000C7D3F302A077D633029027D3C7F0080AA
:107BBF00247D2080127D3E800E7D3CE54975F007C7
:107BCF00A42406800A7D3FE55975F007A42409FF18
:107BDF0064027001FF7E1CED02C6ED7D2080027DE8
:107BEF003FE55B75F009A42416FF7E09ED02C6ED93
:107BFF00C2497E207F00126C3C127B7E7E007F0686
:107C0F00907D1C12C74DE558B4FF01227510007509
:107C1F00A704758307126344E51075F007A42409C0
:107C2F00FFF5177E00E51212C6ED7805EE2404FE6F
:107C3F00E012C6EDD8F67920E030E702792F30490F
:107C4F0017120C8CFAB40408E510700C79658008D3
:107C5F00EA14651070027923E97E1812C6ED7E20B2
:107C6F00E51230E70890936A126C3C8016E511120A
:107C7F007CEA1264FE2010052011028006301203E8
:107C8F00127C9C0510C3E5589510508322127DA4D9
:087C9F00127DBAFD7C00AE1C51
:107CA700AF1B125CEFBE003A8F00C3E57A9513FF56
:107CB700E55E9514FE402B7C007D28125CFCC3EF2B
:107CC70098401F75F0058404FB24F950027B067E5B
:107CD7002CAF170F12D0E10F12D0E10F12D0E10E27
:107CE700DBEF2264B4602464B475F03284C0F01210
:107CF700C6DACE2404CED0E075F00584C0F012C6F3
:107D0700DACE2404CED0E02302C6DA907D18026CC6
:107D17003C2D2D2D000140FFFFFFE0FFFFFFFFC2BD
:107D27005030123F20283CE558F4603720480320A4
:107D37000931D250E559F510303306655860020510
:107D470010127D6E127DCA75A7049006DCE512F04D
:107D5700E511F0E517F0E510F075A7049006E0ECE3
:107D6700F0EBF075A7002275A7047583071263442B
:107D77007813E0F608B819FA9006D07811E6F008FB
:107D8700B819FAE51CF516F0E51BF515F0127DA4F8
:107D97009006DAE514F0E513F075A7002275A7043D
:107DA700758306E51023541E24B0F582E0F513E031
:107DB700F51422120978E5BD2487E5BD923B5002F0
:107DC700249122127DBA75F005A485F012F511E40D
:027DD700F5199C
